:100000000C949B040C94B8040C94B8040C94B8049D
:100010000C94AF140C94B8040C94B8040C94B80469
:100020000C94B8040C94ED050C94B8040C9481065F
:100030000C94B8040C94B8040C94B8040C94B80450
:100040000C94B8040C94B8040C94B8040C94B80440
:100050000C94B8040C94B8040C94B8040C94B80430
:100060000C94B8040C94B804D80B160C290C561137
:100070005611561156115611561156115611561148
:100080005611561156115611561156115611561138
:100090005611561156115611561156112E0C561155
:1000A000560C6A0C850CAD0CDB0CEC0C000D2A0D0B
:1000B000560D560D5E0E5E0E5E0E5E0ED50B9B0E41
:1000C0005F0D760D7E0F880F0910091009100910B9
:1000D0000910561156115611561156115611561136
:1000E00056119D0FF30F09106364696E6F7073757D
:1000F00078585B003C656D7074793E20202020208C
:10010000006572726F723A20777269746520616659
:1001100074657220666F726D61740053494F2D458E
:1001200072726F723A2025690053494F3A434D4429
:100130002054696D656F75740053796E6320576143
:1001400069742E2E2E2020200053746F7070656409
:100150002E2E2E202020003E4E65773C2020202091
:10016000202020004572726F7220696E69742046EB
:1001700041543A20257500252E30386C7820252EE4
:1001800030386C78004572726F7220696E69742025
:1001900053443A202575005344524956452E415444
:1001A00052206E6F7420666F756E6400252E327853
:1001B00020252E327820252E327820252E327820C8
:1001C0002563202575006572726F723A206372652F
:1001D000617465206E65772066696C65000F111388
:1001E00015181A1C1E212325325344726976653175
:1001F0003320206279204B4272006279204B427298
:100200002056312E33005344726976652D4D415886
:100210000053444D58252E34750053444D582568DD
:100220007500415452005446542D49443A20252E1D
:1002300030347800546170652D456D750058313A41
:100240002025692C2058323A2025692C2059313A32
:100250002025692C2059323A2025690020202020B1
:1002600020202020202020200025692066696C6540
:10027000732C20706167652025692F256920202552
:100280007320202020202020202020202000C501B5
:1002900000000000F000180159CE0000FFFF1E0111
:1002A000112059010F00A50050001E0059CE00007A
:1002B000FFFF220168205F010F00CD0050001E00EB
:1002C00059CE0000FFFF2101CA2365019000A5005F
:1002D00050001E0059CE0000FFFF2001AF236B012C
:1002E0009000CD0050001E0059CE0000FFFF1F01FE
:1002F000112070010F002D005A001E0059CE000081
:100300001F052A01E82377010F0055005A001E003F
:1003100059CE00001F052901E8237E010F007D0052
:100320005A001E0059CE00001F052801E823850150
:100330000F00A50046001E0059CE00001F05270132
:10034000E8238A010F00CD0050001E0059CE0000A6
:100350001F052601E82390010F00F5005A001E003A
:1003600059CE00001F052501E8239701A4007D0058
:100370003C001E0059CE0000FFFF240199276B01AD
:10038000A400A5003C001E0059CE0000FFFF230181
:1003900011209C01A4002D003C001E0059CE00003D
:1003A000FFFF31018E21A001A40055003C001E007A
:1003B00059CE0000FFFF30017D21A501A4007D0082
:1003C0003C001E0059CE0000FFFF2F0130206B01C2
:1003D000A400A5003C001E0059CE0000FFFF2E0126
:1003E0001120A801A400CD003C001E0059CE000041
:1003F000FFFF2D019920AD01A400F5003C001E0077
:1004000059CE0000FFFF2C019721C5010F002D00E0
:100410009600F00059CE0000FFFF2B019E26B2018E
:100420000A00C80032001E0059CE000000003A0148
:10043000F61FB6010A002800DB001E0059CE00009E
:10044000000039016B20C6010A005000DB001E00CD
:1004500059CE0000000038016B20D6010A00780058
:10046000DB001E0059CE0000000037016B20E601C2
:100470000A00A000DB001E0059CE0000000036017B
:100480006B20F6015000C80050001E0059CE00003D
:10049000000035010020FC01B300C80032001E003E
:1004A00059CE0000E0073401682000020A00F00085
:1004B00032001E0058540000DFFF330168200402A0
:1004C000B300F00032001E0059CE00001F003201C0
:1004D0005A20C5010A001801E5003F010000000094
:1004E00000002202302641545241545843415343A4
:1004F0004F4D42494E455845584558584644544139
:1005000050494D474241535245414459000000244F
:1005100021E318C318E3180421042100000000009F
:100520000000000000000000000000000004218224
:100530001041084108410861086108456945698220
:10054000108210A210A210C31804210000821041D2
:100550000820002000200041084108456945694104
:1005600008410861084108610882100000821020DB
:100570000020002000200020004108456945694115
:100580000841084108410841086108A21082102072
:100590000020002000200041086108610861086116
:1005A0000861086108610841086108A210A21041B1
:1005B0000820002000410861088210FFFFFFFF00B3
:1005C00000A210A210821061088210A210C318614C
:1005D000084108410882108210FFFF1F001F00FF22
:1005E000FF0000E318A21082108210C318E31882E3
:1005F00010610861088210FFFF1F001F001F001F0D
:1006000000FFFFC318A21082108210C318E31882E3
:100610001082108210A210FFFF1F001F001F001F7A
:1006200000FFFFC318A21061088210C318C318820C
:100630001061088210A210E318FFFF1F001F00FFC7
:10064000FF0000A210821061086108A210821061F0
:100650000841088210C31804212421FFFFFFFF0076
:1006600000C318A21082104108610882101F000008
:1006700000200041088210C318E318E318E318C3F0
:1006800018C318A210610861086108610800000021
:1006900000200041086108A210C318C318A210A2CC
:1006A00010A21082106108410861088210610800E0
:1006B000002000200061088210A210A21082108287
:1006C0001082106108610861088210A210C31861CD
:1006D000084108410861088210A210A2108210820D
:1006E000108210821082108210C3180000000000D7
:1006F00000000000000000000000000000000000FA
:1007000000000000000000000000000000000000E9
:1007100000000000005F00000007000700147F14C5
:100720007F14242A7F2A1223130864623649552233
:10073000500005030000001C2241000041221C0063
:1007400014083E081408083E08080050300000084D
:1007500008080808006060000020100804023E51EC
:1007600049453E00427F4000426151494621414592
:100770004B311814127F1027454545393C4A4949E9
:100780003001710905033649494936064949291E90
:1007900000363600000056360000081422410014CE
:1007A000141414140041221408020151090632499C
:1007B00079413E7E1111117E7F494949363E4141C2
:1007C00041227F4141221C7F494949417F09090952
:1007D000013E4149497A7F0808087F00417F410076
:1007E0002040413F017F081422417F404040407F2C
:1007F000020C027F7F0408107F3E4141413E7F0989
:100800000909063E4151215E7F0919294646494999
:10081000493101017F01013F4040403F1F204020FE
:100820001F3F4038403F63140814630708700807EF
:100830006151494543007F414100020408102000F6
:1008400041417F0004020102044040404040000159
:1008500002040020545454787F48444438384444B7
:100860004420384444487F3854545418087E0901C1
:100870000218A4A4A47C7F0804047800447D4000EE
:100880004080887A007F1028440000417F40007C2F
:10089000041804787C080404783844444438FC2460
:1008A00024241818242418FC7C08040408485454F0
:1008B0005420043F4440203C4040207C1C204020E9
:1008C0001C3C4030403C44281028441CA0A0A07C84
:1008D0004464544C44000836410000007F0000008E
:1008E0004136080010080810087846414678FFFF96
:1008F000FFFFFF426C6F636B2025752020202020B6
:1009000000426175643A202575204C656E677468F5
:100910003A202575204761703A2025752020202037
:1009200000456E64202000426C6F636B20257520AB
:100930002F202575200011241FBECFEFD8E0DEBF89
:10094000CDBF12E0A0E0B1E0EAE7FBE702C005900E
:100950000D92A830B107D9F726E0A8E0B2E001C0B7
:100960001D92A33EB207E1F70E946B110C94BB3DB0
:100970000C9400000F931F9390912102911131C0AC
:10098000E0914001F09141012281338194E1899FFE
:10099000200D311D1124F9017096A591B4918C910F
:1009A00082FF03C00FE110E002C009E51EEC462FF4
:1009B000F9013296849190E032962491622F70E092
:1009C0006B5F7F4F0596413029F0423029F400E0FB
:1009D00018EF02C000EE17E021E043E050E00E9473
:1009E000AB2A1F910F910895CF93DF9340E050E021
:1009F00090E060E3680F71E3E0914001F091410104
:100A00000280F381E02D9F01240F351FF9017096BC
:100A1000C591D491F901A591B49128812B7F2883A8
:100A2000891302C02460288320E3290F11962C9398
:100A30001197823048F0891303C011967C9304C04B
:100A4000913011F411966C939F5F4C5E5F4F95301F
:100A500099F680912102811102C00E941223DF9138
:100A6000CF910895A0E1B0E0E8E3F5E00C94D13433
:100A70006B017C018E010F5F1F4F80E1F801119225
:100A80008A95E9F7C701B601605F7F4F8F4F9F4F8F
:100A90000E94701E611571058105910569F126E9B5
:100AA00032E03A8329834601570124E0B694A794A3
:100AB000979487942A95D1F79C828B82F1E0CF1688
:100AC000F8E0DF06F2E0EF06F10418F020E031E094
:100AD00002C020E830E03E832D830E94D51680E1DD
:100AE000F801A4EBB2E001900D928A95E1F780E065
:100AF0000E94951680E005C086EC91E00E94A0253A
:100B000081E06096ECE00C94ED34E62FF0E0EC54DC
:100B1000FB4F6AE00E941F3480638083906391835F
:100B20000895E4EBF4E08C549B4F1192E817F90719
:100B3000E1F708959091B5059F939091B4059F9327
:100B40001F928F93ECEDF5E083811F928F9382814A
:100B50001F928F9381811F928F9380811F928F9319
:100B60008CEA91E09F938F9388EC95E09F938F930D
:100B70000E948C3788EC95E00E9476268DB79EB750
:100B800040960FB6F8949EBF0FBE8DBF089580E0CB
:100B900090E00E948529E0E7F0E080818160808319
:100BA000E1EBF0E08081876080830895E0E7F0E08A
:100BB00080818E7F80831092B10080912102E0912C
:100BC0004001F091410195E0899FE00DF11D112454
:100BD0000190F081E02D099508951F920F920FB6B4
:100BE0000F921124EF92FF920F931F932F933F9335
:100BF0004F935F936F937F938F939F93AF93BF9325
:100C0000CF93DF93EF93FF93809108028F5F8093E0
:100C100008028F7309F50E945E37EC010E945E376F
:100C20008C0180E090E00E948529C8016CE271E0AF
:100C30000E943F34FC01CE0168E770E00E943F341F
:100C400026E0E22E22E0F22E00E010E028E03CEF69
:100C500042E0BF010E94FB2BFF91EF91DF91CF910A
:100C6000BF91AF919F918F917F916F915F914F91C4
:100C70003F912F911F910F91FF90EF900F900FBE1A
:100C80000F901F9018950F931F9380910D02811163
:100C90001EC0E091BE05F091BF05868981FF09C0A5
:100CA0002FE781E397E1215080409040E1F700C0B9
:100CB00000008BE08093810000EE17E021E043E02C
:100CC00050E065E070E085E090E00E94AB2A81E0B2
:100CD00080930D021F910F9108950F931F9310920F
:100CE000810010920D0200E010E021E043E050E0AE
:100CF00065E070E085E090E00E94AB2A1F910F91C3
:100D000008951F920F920FB60F9211242F933F93C5
:100D10004F935F936F937F938F939F93AF93BF9303
:100D2000EF93FF9380910D02882319F08F5F8093DA
:100D30000D0280910D02853110F00E946D06FF9129
:100D4000EF91BF91AF919F918F917F916F915F9143
:100D50004F913F912F910F900FBE0F901F901895BC
:100D6000A0E0B0E0E6EBF6E00C94D6348CE392E041
:100D70009093BF058093BE0580913802909139020F
:100D8000A0913A02B0913B028093400290934102BD
:100D9000A0934202B0934302E12CF12C60E0C70122
:100DA0000E948C18882309F45CC004EB14E0C1E6AF
:100DB000D0E0F801D1908F01CE010E94733DD8128E
:100DC0004CC02196F4E00F3B1F0799F7E091BE0558
:100DD000F091BF0580819181A281B3818087918745
:100DE000A287B387148615861686178620E130E021
:100DF00040E050E0BA0180E00E94941AC091BE0524
:100E0000D091BF0581E08E8B9091B8048091B90498
:100E1000892B813011F481E28E8B8A899B89AC8980
:100E2000BD89BC01CD0160517109810991091E89FB
:100E300015FD05C020E830E040E050E004C020E0AF
:100E400031E040E050E00E945334213D3240410502
:100E5000510580F010681E8B0DC0EFEFEE1AFE0AF0
:100E60009DCFE091BE05F091BF05168A87E991E01C
:100E70000E94A025CDB7DEB7E7E00C94F234A7E0DE
:100E8000B0E0E5E4F7E00C94CB348091DD0581110E
:100E900055C040E064E070E08CED95E00E94431F97
:100EA000823031F489E291E00E94A0250C94671110
:100EB000AFE7BCE01197F1F700C00000359BFECF13
:100EC000882309F43BC090910F029923B1F01F923F
:100ED0008F938BE191E09F938F9384EB94E09F93AA
:100EE0008F930E948C3784EB94E00E9476260F90BB
:100EF0000F900F900F900F900F908091C205883245
:100F000039F081E09091C105911180E08093C10595
:100F10008091C105882361F0E091C205EB3018F0A3
:100F2000E8EEF1E003C0F0E0E352FE4F849101C02F
:100F300088E690E00E940F1F0C9467111091DD0568
:100F40008091DC059FEC980F943080F42091C005CF
:100F5000813319F42093B6051AC090E030E0205D8B
:100F60003F4F8217930771F481E00FC0813711F072
:100F70000C94671180EB810F843008F0FAC380E392
:100F80008093DC058091DC058F708093B60580919D
:100F9000B605482F50E0B8E18B9FF0011124E45CC6
:100FA000FD4FF093BF05E093BE059689292F297068
:100FB00011F40C946711133509F40AC1292F2B7F02
:100FC000268B123209F4DCC018F4113241F000C152
:100FD000103509F4F9C0173509F4F6C0F9C080914D
:100FE000BD05813019F40091E70501C000E093FFD1
:100FF00029C081E40E94281F62E08091B6050E940A
:10100000BA040E9443060023C1F08091E5058111D6
:1010100005C060E87EEC82E090E0C2C0813041F023
:10102000E091BE05F091BF0586898460868BEDC096
:1010300060E87EE985E090E0B3C060E078E681E0BA
:1010400090E0AEC094FF07C0C12C78E6D72EEE2406
:10105000E394F12C07C060E1C62E68E6D62EEE249C
:10106000E394F12C8330E1F2811111C088E1849F77
:10107000F001859FF00D1124E45CFD4F8289938976
:10108000A489B589C816D906EA06FB0649F60111F6
:1010900003C000E810E002C000E011E01092BD05BE
:1010A000E091BE05F091BF05878980FDB9CF8689A3
:1010B00086FDB6CF83FF03C0877F868B08C081E49F
:1010C0000E94281F62E08091B6050E94BA0480E069
:1010D00091E00E949105E091BE05F091BF058689DF
:1010E00084FF04C0812C912C54011CC050E1852E3A
:1010F000912CA12CB12C16C0E1E0CE16DE06E10445
:10110000F10420F0C12CD12C7601D3949601B501C5
:10111000A40181E00E94941A892B99F08C0C9D1CEB
:10112000AE1CBF1CE091BE05F091BF05C288D388FC
:10113000E488F588C818D908EA08FB08E9F680E0D1
:1011400001C081E0E4EBF4E098012C543B4F9FEFA9
:101150009193E217F307E1F7882379F01092B40432
:101160001092B504E091BE05F091BF0586898460B8
:10117000868B81E091E00E94A02540E0B801D8C6AE
:1011800093FF1FC081E40E94281F62E08091B60592
:101190000E94BA040E94430660E078E082E090E09A
:1011A0000E94320581113CCF1091B605E091BE0539
:1011B000F091BF05808991899093DF058093DE05CA
:1011C0004AC727FF2DCF65CF62E00E94BA0426C030
:1011D00061E00E94BA048091DD059EEA980F92308A
:1011E00050F4E091BE05F091BF05968993FF16C0BB
:1011F000833529F413C08E3489F08F3479F08F331E
:1012000021F48091C205883249F480910F0288232D
:1012100009F4C6C38EE40E949A05C2C381E40E9409
:10122000281F8091700080FD0E94D6058091DD0509
:10123000803509F408C158F48E34B1F008F0A0C02C
:101240008F3311F00C9467118091C20529C3833547
:1012500009F45DC2873509F4F6C0823511F00C94AB
:1012600067110E944306EFC0E090BE05F090BF05F5
:10127000D70152964D905D906D907C905597569603
:101280008C9183FF0BC09091BD05913009F472C021
:10129000412C38E6532E66246394712CB82FB07419
:1012A000BD8385FF03C000E011E002C000E810E04C
:1012B000C12EDD2480E090E053014201E0E88E225F
:1012C00021EE35E03C832B831C013CE0230E311CD6
:1012D000DC011196BF83AE830E94733DEB81FC81DC
:1012E0008193FC83EB838E819F812816390681F7D9
:1012F000FD81F11113C08091E9059091EA05A0915B
:10130000EB05B091EC0588159905AA05BB0531F4EC
:101310008091E70590E08C159D0561F1C101209158
:10132000E105213069F6C092E7050093E8052D81BB
:10133000222341F03DE2430E34EB531E611C711C2D
:101340000DE710E0D70156968C9185FF06C0B0E8F6
:101350004B0EB1E05B1E611C711C980140E050E037
:10136000C301B2010E9453343093E3052093E40596
:101370004093E50540E06CE070E081EE95E0DAC571
:101380006CE070E081EE95E00E948A1F81119FC79A
:101390000091BE051091BF05D8015696EC91569765
:1013A000F091E705E3FF09C0FF2311F0E06202C0FE
:1013B000EF7DD8015696EC9342C02091E505822F2F
:1013C00090E0A0E0B0E09C01AD012F5F3F4F4F4F98
:1013D0005F4FA091E105B0E00E94B8349B01AC01E1
:1013E000A091E305B0E0BA2FAA278091E405A80FE9
:1013F000B11D0E94C3349B01AC01AF2FB0E0BA2FE6
:10140000AA278091E805A80FB11D0E94C334E4FD0E
:1014100004C0605F7F4F8F4F9F4FE5FF04C060584F
:10142000714081099109F80102891389248935895C
:10143000601771078207930711F083E001C081E014
:101440008093BD0523C780E890E09A83898310923A
:10145000BD05C090DE05D090DF05C114D10409F4AC
:1014600052C1E091BE05F091BF05E689E6FD73C06B
:10147000E1FF15C090910E028091B605981731F0EA
:101480000E944A2F8091B60580930E0242E051E0FF
:10149000BE016F5F7F4FC6010E94C42F3DC0F4E0C4
:1014A000CF16D10458F421E0C21AD108D694DC2C0E
:1014B000CC24D794C794E12CF12C1CC0E5FF03C0C9
:1014C000A0E0B1E002C0A0E8B0E0BA83A983A60121
:1014D00060E070E09A01AB012450310941095109E3
:1014E0000E94B8346B017C0130E8C30E31E0D31E9A
:1014F000E11CF11CE4FD05C080E1C80ED11CE11C1B
:10150000F11C8091DD0529813A81823549F4B701CA
:10151000A60180E00E94941A892B09F4F4C0F0C05F
:10152000B90184EB94E00E948A1F8111D0C60E9409
:101530004306E091BE05F091BF05878980FDE3C0B9
:1015400029813A81B701A60181E00E94941A892B72
:1015500009F4D9C09BC68091DD05823551F060E861
:1015600070E084EB94E00E948A1F882309F4CBC0CA
:10157000AEC680E890E00E94910594E0C916D104BF
:10158000F0F0E090BE05F090BF05F70182899389E5
:10159000A489B589BC01CD0164587F4F8F4F9F4FFF
:1015A0002DE730E040E050E00E94533449015A01F9
:1015B0008901F8E6CF16F1E0DF0629F574C0C6010F
:1015C0009695982F882797958795835190402091DD
:1015D000C30577E0972E920E04EB14E07C0120E81F
:1015E000E20EF11C5C013FEFA31AB30A0E94733DA7
:1015F000873009F4892DD8018D938D01C501AE1472
:10160000BF0481F7BECFB9E6CB16B1E0DB0609F027
:101610004FC060E0F701808991890E948C18A4EB8B
:10162000B4E080E090E030E22D914FEB420F4A3180
:1016300020F040ED420F4A3030F4E82FF0E0EC5457
:10164000FB4F20838F5F973011F09A3049F4981741
:1016500038F0E82FF0E0EC54FB4F30838F5FF7CF8A
:101660009F5F9B3009F7EFEBF4E08291858324E0E4
:10167000E43BF207D1F7E4ECF4E084E395E08E1765
:101680009F0711F01192FBCF003932E0130710F0E1
:1016900086E401C082E48093B40481E791E09093F2
:1016A000B8048093B7049092B6048092B50424C025
:1016B00081E7C81681E0D806F8F09601ADE7B0E002
:1016C0000E94A234AB01BC014D52544B6109710917
:1016D0002DE730E080E00E94941A8D37910520F0CC
:1016E00096012F5F3F4F02C020E030E0309331057C
:1016F000209332058093330580E890E09A838983B4
:1017000069817A8114C469817A8141E011C4909120
:101710000D02911190E19093B404E091BE05F09117
:10172000BF05868987FF03C090689093B40485FF46
:1017300005C09091B40490629093B40482FF07C0F6
:101740009091B40494609093B4048B7F868B8789C6
:1017500080FF05C08091B40488608093B4048091B8
:1017600002018093B50480EE8093B6041092B70412
:10177000ADC081E40E94281FE091DD05EB3D09F436
:101780008AC01F7088EF95E09093BF058093BE05D7
:101790008E2F90E0FC01E05CF109E034F10508F0E7
:1017A00085C5EC5CFF4F0C94943400E010E0B2C2AD
:1017B00080E091E00E9491058091DE059091DF0527
:1017C00000EC14E06C01A5E1CA0ED11C7C01BFEF56
:1017D000EB1AFB0A60E00E948C188823D9F0EC1405
:1017E000FD0429F48091B404F801808313C0A4EBB4
:1017F000B4E0C8010B96F8012D912193E817F90781
:10180000D9F78091B805D8011B968C93045F1F4FC0
:10181000C701DCCFE4EBF4E084858193B5E0E53AE1
:10182000FB07D1F740E061EF70E082C38091DE05F5
:101830008A3F08F03BC58093C2051092C105EFE7CF
:10184000FCE03197F1F700C0000083E40E94281FFC
:101850005FCB8091DE058093C30518C583E292E0DB
:10186000A4EBB4E04DEC54E0FC012191CF012D93A9
:10187000F4E0AD3CBF07C1F7A8EFB5E085EE94E01A
:101880002D91FA012193AF018E179F07C9F740E010
:1018900061E370E04DC3E091BE05F091BF0586891C
:1018A0008093B40440E061E070E042C36091DE05E3
:1018B0007091DF0580E090E00E9407176093B40408
:1018C0007093B5048093B6049093B70440E064E04D
:1018D00070E02EC364E070E084EB94E00E948A1F05
:1018E0008111F5C46091B4047091B5048091B6047F
:1018F0009091B7046093C4057093C5058093C605A5
:101900009093C7050E94D516C1C46091C40570911B
:10191000C5058091C6059091C7050E94D5168FE731
:101920009CE00197F1F700C0000083E40E94281FAB
:10193000AFE7BCE01197F1F700C0000060E072E093
:1019400084EB92E00E94001F182F60E072E084EBAD
:1019500092E00E942F1F812FB8C46091C40570913E
:10196000C5058091C6059091C7050E94D51640E235
:1019700060E072E084EB92E00E94431FEFE9FFE039
:101980003197F1F700C00000882361F06091C40531
:101990007091C5058091C6059091C7050E94D51626
:1019A0008EE493C481E40E94281F80E00E94951673
:1019B00081117CC46BC46091DE05662309F466C4A2
:1019C000E9EEF1E0A4EBB4E080E094919D938F5FA9
:1019D00031966813FACFAAC20E94CC168091DE0518
:1019E000882319F00E94B0065FC48FE79CE001973E
:1019F000F1F700C0000083E40E94281F0C9400004F
:101A00009091DE05953008F051C4A8E19A9FF0014D
:101A10001124E45CFD4F868983FD02C08E7F01C0E6
:101A2000867F868BE0914001F09141010280F38135
:101A3000E02DB4E19B9FE00DF11D1124859194915F
:101A40004CE050E064EF70E003960E946E378091A6
:101A5000C0055BC2E091DE05E53008F027C428E14F
:101A6000E29FF0011124E45CFD4F868980FD08C0EF
:101A70008EE090E00E94910540E06EE070E058C278
:101A8000F093BF05E093BE0584819581A681B7815F
:101A90008093FC059093FD05A093FE05B093FF0590
:101AA000908981899093DE058093DF0560E08091C5
:101AB000DE059091DF050E948C18082F3CC06BE07A
:101AC00070E08DEE95E00E948A1F811100C4809124
:101AD000DF05882309F4DAC31091DE05812F806FBA
:101AE0008093DD051092DF051092DE05E090DE05A3
:101AF000F090DF058091DD05803F08F0B5C160E022
:101B0000C7010E948C18882309F4F2C1EDEEF5E0BC
:101B1000A4EBB4E081918111C1C1119635E0E83F99
:101B2000F307C1F78091DD05803F08F0BCC183EE6B
:101B30008093DD0501E02091B8052093BF048091DA
:101B4000DD05833E61F4E091BE05F091BF0580891B
:101B500091899093C1048093C0041EE0A7C0853E84
:101B600009F0A3C0A091BE05B091BF0552964D915A
:101B70005D916D917C9155974093C0045093C10441
:101B80006093C2047093C3048091B905D090BA05E4
:101B90008093C404D092C5048091BB059091BC058C
:101BA0009093C7048093C604E8ECF4E086EE94E0DA
:101BB00030E231938E179F07E1F752966D917D9138
:101BC0008D919C915597287119F420E32093D104AD
:101BD00044EBE42E44E0F42E1AE05AE0852E912CDA
:101BE000A12CB12C611571058105910551F0A5015C
:101BF00094010E9453346063D7015D966C93B901E0
:101C0000CA011150B1E0EB1AF1081111EBCF8DE2CE
:101C10008093D7048093DA048AE38093E00480936E
:101C2000E3048D2D869590E08454984F64E670E02F
:101C30000E942B34962F182F6FE1892F0E94850563
:101C400061E2812F0E9485058091B9059091BA05C6
:101C500025E0969587952A95E1F764E28F700E94BA
:101C600085058091B90567E28F710E948505809195
:101C7000BC056AE28695869586950E9485058091C9
:101C8000BB059091BC0535E0969587953A95E1F7AF
:101C90006DE28F730E9485058091BB058F7160E3B3
:101CA000880F0E94850512E301C01CE0011104C0E9
:101CB00082E390E00E949105612F38C161E080913C
:101CC000DE059091DF050E948C18811106C080E02E
:101CD00090E0FC01EC54FB4F09C0E4EBF4E080E041
:101CE00090E0019621912111FCCFF3CFCF01845BCD
:101CF00094408F3F910509F010F41192F7CF809135
:101D0000DD05865E60E071E002C0759567958A9595
:101D1000E2F70DC160E0C8010E948C18882319F019
:101D20000F5F1F4FF7CF1093B5040093B40440E04A
:101D300062E070E0FDC08091DE058150843118F0D2
:101D400084E18093DE050091DE058090FC05909093
:101D5000FD05A090FE05B090FF0510E08FE2D82EA3
:101D600060E080E090E00E948C18E091BE05F09168
:101D7000BF05882309F450C08091B80584FF4CC08A
:101D80008091B4048E3209F047C08091B5048E3240
:101D900009F042C0011107C0A12FB0E0AC54BB4F05
:101DA0008FE38C9339C001504480558066807780E2
:101DB00080819181A281B38184839583A683B78337
:101DC000E12CF12C60E0C7010E948C18882341F2BD
:101DD000E091BE05F091BF0580819181A281B38120
:101DE000481659066A067B0699F41C50E12FF0E06C
:101DF000DF01AC54BB4FDC92A4EBB4E0EB54FB4FDF
:101E0000CF010B962D9121938E179F07D9F7A8CF5D
:101E1000EFEFEE1AFE0AD6CF84829582A682B782B1
:101E2000812F90E0DC01AC54BB4F119520E03D9137
:101E3000E22FF0E0EC54FB4F30832F5F2113F7CFFC
:101E40008195811103C01092B40481E0E82FF0E085
:101E5000EC54FB4F10828F5FC9F76091DE05FCE008
:101E60006F9FB001112463C0153008F048CE28E1FF
:101E7000129FF0011124E45CFD4FF093BF05E09345
:101E8000BE058091FC059091FD05A091FE05B091E5
:101E9000FF0584839583A683B78331CE9C918917F0
:101EA00009F43BCE21C01530D0F488E1189FF00131
:101EB0001124E45CFD4FF093BF05E093BE058091D3
:101EC000FC059091FD05A091FE05B091FF0584836E
:101ED0009583A683B78360E0C7010E948C18F092B7
:101EE000DF05E092DE05B7C09FEFE91AF90A07CED9
:101EF0008091DD05803F08F0D9C1BACD8091DE0523
:101F0000853008F081E08093C0050E94F404BEC1D2
:101F10006091DE05E091DF05F0E0E054FA4FA4EBBC
:101F2000B4E0862F91919D938150E1F770E040E0FD
:101F300084EB94E00E94C01FCAC160E080E090E0A2
:101F40000E948C18811116C08091DE05882309F447
:101F50009DC1E091BE05F091BF058091380290913E
:101F60003902A0913A02B0913B0284839583A68303
:101F7000B7837ECD8091B80584FFE6CF8091B4040D
:101F80008E3211F78091B5048E32F1F6E091BE05E4
:101F9000F091BF05C480D580E680F7808081918173
:101FA000A281B38184839583A683B7838091DE0564
:101FB000882351F200E010E060E0C8010E948C1814
:101FC000882311F2E091BE05F091BF0580819181D7
:101FD000A281B381C816D906EA06FB0609F4A7CD8B
:101FE0000F5F1F4FE9CF8091380290913902A09185
:101FF0003A02B0913B028093FC059093FD05A093BB
:10200000FE05B093FF0560E080E090E00E948C1830
:102010003DC11530B0F4A8E11A9FF0011124E45C31
:10202000FD4FF093BF05E093BE058091FC059091B4
:10203000FD05A091FE05B091FF0584839583A683DD
:10204000B78360E08091DE059091DF050E948C18D7
:10205000882309F42BC19091B805E091BE05F09159
:10206000BF0594FF09C080819181A281B3818483DF
:102070009583A683B78301C14081518162817381B9
:102080004087518762877387148615861686178660
:1020900086898870868B90FD02C0178A02C081E015
:1020A000878B8091BC04813409F049C08091BD04C4
:1020B000843509F0B1C08091BE04823509F0A1C019
:1020C00020E130E040E050E0BA0180E00E94941A44
:1020D000E090BE05F090BF05F7018689982F9160CA
:1020E000968B2091B8049091B904922B913011F401
:1020F0008162868BF70182899389A489B589BC01A5
:10210000CD016051710981099109D688D5FE05C0BC
:1021100020E031E040E050E004C020E830E040E062
:1021200050E00E945334213D32404105510508F4EE
:102130007AC08D2D8068D70156968C9374C08835EF
:1021400059F48091BD04863409F066C08091BE04C4
:10215000843409F061C01AC0833459F48091BD04FD
:10216000813409F059C08091BE04833509F054C010
:102170000DC0823409F050C08091BD04893409F04B
:102180004BC08091BE048E3409F046C024E030E09C
:1021900040E050E0BA0180E00E94941A8091B404BB
:1021A000863469F48091B504853579F48091B6045C
:1021B0008A3459F48091B704893439F42DC08F3FA3
:1021C00021F48091B5048F3F39F1E091BE05F09183
:1021D000BF058689982F9161968B428953896489BE
:1021E00075894130B8E65B07B1E06B077105D8F03F
:1021F000413058406240710510F4816913C0816319
:1022000011C0883549F40E944A2FE091BE05F09133
:10221000BF058689836006C0E091BE05F091BF05C9
:102220008689816C868B8FEF810F843030F560E07A
:102230008091DE059091DF050E948C1884EB94E07C
:102240000E948E20E0914001F09141010280F381D3
:10225000E02D34E1139FE00DF11D1124859194913F
:102260004CE050E064EB74E003960E947D3780916F
:102270002102811102C00E941223E091BE05F0915B
:10228000BF05868983FF02C00C94470880910F0226
:10229000882321F083E40E949A0506C08FE79CE022
:1022A0000197F1F700C0000083E40FC080910F0296
:1022B000882321F085E40E949A0506C0AFE7BCE0C0
:1022C0001197F1F700C0000085E40E94281F2796AF
:1022D000E2E10C94E734A4E0B0E0E1E7F1E10C9432
:1022E000CB34459A3D9882E08093680080E28093E9
:1022F0006C0080B7846880BF8FE080937E0083B5D8
:10230000816083BD84E79BEC909389008093880073
:1023100080916F00826080936F001092C1051092CF
:10232000C3051092C0051092B6051092BD0580E657
:1023300090E00E94733D8093C2050E944C27E0917B
:102340004001F09141010190F081E02D09958091CB
:102350003F0182FF03C081E08093C00588E690E0E2
:102360000E940F1F61E08091B6050E94BA040E948E
:1023700027152FEF31EE44E0215030404040E1F787
:1023800000C000000E946D158823E1F11F928F9319
:1023900085E891E09F938F9384EB94E09F938F93D4
:1023A0000E948C3784EB94E00E9476268091BB02D9
:1023B0008F938091BA028F938091B9028F9380910D
:1023C000B8028F938091B7028F938091B6028F935A
:1023D0008091B5028F938091B4028F9387E791E04B
:1023E0009F938F9324EB34E03F932F930E948C377D
:1023F00084EB94E00E9476260FB6F894DEBF0FBE01
:10240000CDBF7AC08DB581608DBD8CB58D7F8CBD03
:102410008CB58E7F8CBD1092520210926A0210927F
:10242000820210929A021092B2020E9439178823F7
:10243000B9F01F928F9384E691E09F938F9384EB82
:1024400094E09F938F930E948C3784EB94E00E94DA
:1024500076260F900F900F900F900F900F904CC01A
:1024600089E08093210266E9E62E61E0F62E91E094
:102470009B83C7010E947B3D6093FC057093FD0523
:102480008093FE059093FF056F3F7F4F8F4F9F4FC7
:1024900089F0C70104960E94813D9093DF058093E7
:1024A000DE058B81806F8093DD05F1E7F093DC051D
:1024B0000E943F072B812F5F2B8336E0E30EF11C38
:1024C0002530B9F6109221020E9412238091380221
:1024D00090913902A0913A02B0913B028093FC05A1
:1024E0009093FD05A093FE05B093FF050E94B006F2
:1024F0008091C0050E94F40460E08091B6050E94BE
:10250000BA047894612C712C44EB54E05C834B83C7
:10251000212C312C210158E1852E0E94C72D8823C2
:1025200009F45AC18091700080FF03C00E94D60553
:102530003EC10E942128009709F446C1109224064A
:10254000FC017096259134913C832B833A83298337
:10255000FC01C590D4907601F89448EF55E0509373
:10256000BF054093BE0520912102211116C0F6013E
:102570002081243491F4E0914001F09141012281C5
:102580003381AC01421B530B9A0135952795359544
:1025900027955DEC259F902C1124FC0172962591C6
:1025A0003491F90109958C0178948091C0059816B1
:1025B00079F0EB81FC81808182FF0AC09092C00596
:1025C000911002C00E94B0068091C0050E94F404E0
:1025D000F60180818E33A9F4899CF0011124E45C1A
:1025E000FD4F008911890F5F1F4F84819581A6815E
:1025F000B781E091BE05F091BF0584839583A683E2
:10260000B78301151105F9F0F8940F3FFFEF1F078D
:1026100031F422EE2093DD059092DE050EC0899CF8
:10262000F0011124E45CFD4F168A892D806F8093A0
:10263000DD051093DF050093DE0531E73093DC05FF
:102640000E943F07789480912102811128C0F601F1
:1026500080818E3421F58091C005882301F1889E08
:10266000F0011124E45CFD4F96899860968BE0910F
:102670004001F09141010280F381E02D24E1829F2D
:10268000E00DF11D1124E590F4904CE050E067E579
:1026900071E0C70103960E946E370E941223809159
:1026A0002102833009F073C0F7018081833509F07E
:1026B00073C0E0914001F09141010188F289E02D61
:1026C000B496A591B4918091B70580FD03C08C911B
:1026D00082FF21C08091B7058E7F8093B705EB8183
:1026E000FC8180818B7F80838C918B7F8C9329E40C
:1026F000E22E21E0F22E0AE812E520EE3FEF42E062
:1027000064E870E083E290E00E94FB2B0E941223B9
:10271000612C712C41C0E091BE05F091BF05808114
:102720009181A281B38180879187A287B3870E941C
:10273000C7328091B70581608093B705EB81FC813A
:1027400080818460808399E3E92E91E0F92E0AE884
:1027500012E520EE3FEF42E064E870E083E290E0B3
:102760000E94FB2B0E9412238091B70581FD19C0A6
:10277000FAEA26EE36E941E0F15020403040404090
:10278000D9F7000084EB94E09C838B830EC0E4EBCC
:10279000F4E0FC83EB8309C024EB34E03C832B831F
:1027A00004C044EB54E05C834B8300E21EE40E94CF
:1027B000C72D8111FCCF5FEF80E792E05150804040
:1027C0009040E1F700C000001092090210920A0246
:1027D00010920B0210920C028091B70580FF24C06A
:1027E000F8948091B70581FF04C0C3010E94FA32BA
:1027F00003C0C3010E940F323C01892B21F080915C
:10280000B70580FD10C088E690E00E940F1F809100
:10281000B7058E7F8093B705E981FA8180818B7F30
:1028200080830E941223789480913F0181FF5AC0D7
:1028300080912102813009F055C0F0902406FF20DC
:1028400009F450C00032FEE41F0709F049C023E13B
:102850002F1518F01092240602C083E1F82E409143
:102860003B0150913C0141505109A12CB12CC12C8C
:10287000D12CE12C01E02AE130E06AE070E085E053
:1028800090E00E94562ACF2CEB80FC8000E010E004
:1028900020EE3FEF42E06AE070E085E090E00E94C9
:1028A000432C4B815C8184E0443B580769F0FA017A
:1028B00001900020E9F7CF0144978417950739F478
:1028C000E3EBF4E0FC83EB8302E21EE402C000E0F1
:1028D00010E02B813C812F5F3F4F3C832B8302C054
:1028E0000E5F1F4F31EA231630EF330639E14306FE
:1028F000510430F00E94CC16212C312C210105C04E
:102900004FEF241A340A440A540A80913F0184FF8D
:1029100004CE80912102811100CE80910902909114
:102920000A02A0910B02B0910C02813854E895077D
:102930005EE1A507B10538F0809170008111EDCD01
:102940000E94C705EACD0196A11DB11D8093090221
:1029500090930A02A0930B02B0930C02DECD1F925B
:102960000F920FB60F9211242F933F934F935F93C3
:102970006F937F938F939F93AF93BF93EF93FF9347
:10298000359929C080910001909101019093BF0574
:102990008093BE05109224061092DD050E943F0729
:1029A00060E08091B6050E94BA048091BE059091C6
:1029B000BF05909301018093000188EF95E090930B
:1029C000BF058093BE051092090210920A02109270
:1029D0000B0210920C02FF91EF91BF91AF919F916A
:1029E0008F917F916F915F914F913F912F910F90B8
:1029F0000FBE0F901F9018952A9A229A2D9A259A09
:102A00002498239A8DB58E7F8DBD83E58CBD8DB5C1
:102A100008958EBD0DB407FEFDCF8EB508958FEFDE
:102A20000E9409150895FB01E40FF51F39E06E17A8
:102A30007F0761F0229198E0880F482F422747FDD9
:102A40008327220F9150C1F78F77F1CF08950E940D
:102A5000FC140895A5E0B0E0E0E3F5E10C94DA346D
:102A60004A835B836C837D83806489830E9409151C
:102A70008D810E9409158C810E9409158B810E940D
:102A800009158A810E94091541E050E0BE016F5F7F
:102A90007F4F80E00E94131544E050E0BE016E5F5E
:102AA0007F4F0E941315880F81600E9409151FEF48
:102AB0000E940F15115011F087FDFACF2596E3E023
:102AC0000C94F634CF932A980E942A15C82F2A9A7C
:102AD0000E940F158C2FCF910895EF92FF920F93C4
:102AE0001F93CF93DF938FEF9FEFDC01809311064D
:102AF00090931206A0931306B09314061092150635
:102B0000809110068E7F80931006CAE00E940F15F8
:102B1000C150E1F7DAE040E050E0BA0180E00E9405
:102B20006215813031F0D150B1F78093B402C1E029
:102B300091C084EBE82E82E0F82E1AE02A984AEA47
:102B400051E060E070E088E00E942A15D82F8130C3
:102B5000C1F4870184E0E80EF11C0E940F15F80112
:102B600081938F01EE16FF06C1F78091B602813086
:102B700031F48091B70210E08A3A11F402C010E0FB
:102B8000D6E02A9A0E940F158D2F8B7F813061F03D
:102B90008FEF810F112311F0182FD0CFD63020F0F6
:102BA000F701D083C2E056C00FEF13E040E050E0E1
:102BB000BA0187E30E946215D82F8230A8F540E061
:102BC00050E060E070E489E20E946215811127C044
:102BD0002A9840E050E0BA018AE30E942A15D82FD3
:102BE0000E940F158093B8020E940F158093B902BE
:102BF0000E940F158093BA020E940F158093BB02AA
:102C00002A9A0E940F158091B80286FB882780F9C6
:102C10009091100680FB90F99093100605C001502A
:102C2000110921F6C3E016C0D53041F440E050E070
:102C3000BA0181E00E94621581110BC040E052E0B0
:102C400060E070E080E10E946215882319F0C5E021
:102C500001C0C4E08C2FCDB7DEB7E6E00C94F334AE
:102C6000CF93DF93AB01BC012A988091100680FDC1
:102C700007C089E0440F551F661F771F8A95D1F75B
:102C800081E10E942A15811115C00E940F158E3F07
:102C9000E1F7C4EBD2E00E940F15899384E0C43BB6
:102CA000D807C9F70E940F150E940F152A9A0E9493
:102CB0000F1580E0DF91CF910895CF93DF93AB01A3
:102CC000BC012A988091100680FD07C089E0440F5E
:102CD000551F661F771F8A95D1F788E10E942A1534
:102CE000811120C00E940F158EEF0E940915C4EBC0
:102CF000D2E089910E94091584E0C43BD807C9F746
:102D00000E940F150E940F150E940F15982F9F719A
:102D1000953041F40E940F158823E1F32A9A0E940E
:102D20000F1580E0DF91CF9108950F931F93CF93FC
:102D3000C82F00E018EF21E043E050E065E070E0CC
:102D40008FE090E00E94AB2ACC23F1F0C0E16091CB
:102D500011067091120680911306909114060E943C
:102D60005D16882319F0C15091F7FFCF1092150618
:102D700000E010E021E043E050E065E070E08FE02B
:102D800090E00E94AB2A03C081E08093150680E0AA
:102D9000CF911F910F91089580911506882321F0FE
:102DA00081E00E949516FACF0895CF92DF92EF92BC
:102DB000FF92CF93C0901106D0901206E0901306B8
:102DC000F0901406C616D706E806F90611F48FEF40
:102DD00018C06B017C010E94CC16C0E0C701B6018F
:102DE0000E943016C150882319F0C111F7CFEFCFE0
:102DF000C0921106D0921206E0921306F0921406C9
:102E000080E0CF91FF90EF90DF90CF900895CF9228
:102E1000DF92EF92FF92C0902F02D0903002E090AC
:102E20003102F0903202611571058105910569F456
:102E30008091330290913402A7019601281B390B2F
:102E400041095109CA01B9010FC09B01AC012250CF
:102E5000310941095109A0913702B0E00E94B8340C
:102E60006C0D7D1D8E1D9F1DFF90EF90DF90CF900C
:102E70000895A0E0B0E0EFE3F7E10C94CD3460E01A
:102E800070E0CB010E94D5168111E8C0D091760484
:102E900080907A0490907B04A0907C04B0907D0494
:102EA000C501B4010E94D516C82F8111D9C0E09187
:102EB000C502F091C60284E0F695E7958A95E1F7A0
:102EC000F0933402E09333028091CA029091CB02D6
:102ED000009719F0A0E0B0E008C08091D80290916E
:102EE000D902A091DA02B091DB0280932B02909379
:102EF0002C02A0932D02B0932E02C090C202D0905B
:102F0000C302E12CF12CA091C40220912B0230913C
:102F10002C0240912D0250912E02B0E00E94B83454
:102F20002B013C01B501A4014C0D5D1D6E1D7F1DE3
:102F30008F0120E030E0D301C201840F951FA61F4E
:102F4000B71F800F911FA21FB31F80932F02909372
:102F50003002A0933102B09332028091C702909167
:102F6000C802009719F0A0E0B0E008C08091D40238
:102F70009091D502A091D602B091D70284199509FB
:102F8000A609B7098C199D09AE09BF09801B910BD1
:102F9000A20BB30B8093230290932402A0932502EB
:102FA000B09326028091C102809337028091BF02C4
:102FB0009091C0029093360280933502409327028D
:102FC000509328026093290270932A028FEF9FEF9B
:102FD000DC018093160690931706A0931806B09311
:102FE0001906DD3038F4DB3098F4D43029F0D630CF
:102FF000C9F502C0DE30B1F5E091BE05F091BF0524
:103000001482158216821782809110068D7F13C05C
:103010008091E0029091E102A091E202B091E3027E
:10302000E091BE05F091BF0584839583A683B783A5
:1030300080911006826080931006E091BE05F091A9
:10304000BF0584819581A681B781809338029093D2
:103050003902A0933A02B0933B0205C0C1E003C01D
:10306000C2E001C0C3E08C2FCDB7DEB7E0E10C9425
:10307000E9348F929F92AF92BF92CF92DF92EF92FC
:10308000FF922091100621FF0EC042E0660F771FCD
:10309000881F991F4A95D1F7CC24CA94DC2CEC2CBC
:1030A0005FE0F52E09C0660F771F881F991FCC249B
:1030B000CA94DC2CE12CF12C20913502309136029F
:1030C00040E050E00E9453344B015C0180912702A4
:1030D00090912802A0912902B0912A02BC01CD0151
:1030E000620F731F841F951F0E94D516F401EC54C4
:1030F000FD4F80819181A281B381BC01CD016C2102
:103100007D218E219F21FF90EF90DF90CF90BF9087
:10311000AF909F908F900895AAE0B0E0E2E9F8E1C7
:103120000C94CB341C016A83E091BE05F091BF057D
:10313000C480D580E680F7808091160690911706AE
:10314000A0911806B0911906C816D906EA06FB0622
:1031500051F0C0921606D0921706E0921806F0922F
:10316000190610921A0680911A06882389F0209178
:103170001A0230911B023E832D832215330598F0ED
:103180002215330529F4813019F43A81332359F09B
:10319000C701B6010E9407172B013C0110E01E82F7
:1031A0001D82198240C000911002809016029090FA
:1031B0001702A0901802B0901902C0901102D0908E
:1031C0001202E0901302F09014021091150219827D
:1031D000240135018FEF481A580A680A780AC50198
:1031E000B4010E94D51690E2099FF0011124EC541D
:1031F000FD4F4081442309F4E9C0453EC9F4B0962F
:103200000F5F0031B1F7C114D104E104F10409F0FA
:10321000CCC0812F90E0209133023091340282178C
:10322000930708F0BBC01F5F5301420100E0D0CFFD
:1032300083858F3009F053C0AA81AA2301F3842F1C
:1032400090E001978F709927BDE0B89FB001B99FBA
:10325000700D11246C547B4F9F017A876987CF01D1
:103260000A969C838B83F887EF83AF81B88511968C
:103270005C91A985BA855D93BA87A9878F81988566
:10328000029698878F83AB81BC818A179B0769F769
:10329000CB0105969C838B83CF010C96D9011E969A
:1032A0005C91AB81BC815D93BC83AB832E5F3F4F50
:1032B0008217930799F7848DDB011B968C931B97DC
:1032C000868D1C968C931C9746FF02C01D961C92FF
:1032D0004F70413009F093CF31E0398390CFB981FD
:1032E000BB2361F02D813E812215330509F470C0A6
:1032F0002F5F3F4F3E832D83198281CF4E3229F4B9
:103300009181903211F484FD7ACF83FD78CF8D8145
:103310009E8182159305D9F5CF0164EB74E0AB0172
:10332000DC012D91CD01DA012D93AD01B4E04F3BCD
:103330005B07B1F71092BF042A81222309F44AC027
:103340001092C0048091BE048093BF048091BD049C
:103350008093BE048091BC048093BD048091B4042A
:103360008E3219F08EE28093BC0424EB34E0DB0152
:103370008D91BD01803221F0D9018C932F5F3F4F99
:10338000DB018C918111F3CFD9011C9223C02D81D7
:103390003E812F5F3F4F3E832D8331CF90911006AA
:1033A000892F827091FD3FCF6EC080913702181730
:1033B00008F439CFC701B6010E9439186B017C01AE
:1033C0000E9407172B013C0110E02DCF80E005C0C3
:1033D00082E003C03E822D8281E0A091BE05B091C3
:1033E000BF054489558960E070E0BA01552744273C
:1033F000228D338D2901612C712C44295529662990
:1034000077294D935D936D937C93139751963C92DE
:103410002E925097448D558D668D778D52964D9393
:103420005D936D937C93559793859093B80526890A
:1034300037893093BC052093BB05208D318D3093A7
:10344000BA052093B9058823E9F0AD81BE81B09318
:103450001B02A0931A02009310028092160290920F
:103460001702A0921802B0921902C0921102D092D3
:103470001202E0921302F09214021093150280934C
:103480001A0601C080E02A96E2E10C94E734A0E03D
:10349000B0E0EDE4FAE10C94D5346B017C01E091ED
:1034A000BE05F091BF0584859585A685B785C816AC
:1034B000D906EA06FB0660F480819181A281B3817E
:1034C00080879187A287B38714861586168617860C
:1034D000C091BE05D091BF050C851D852E853F8509
:1034E000688579858A859B85C016D106E206F30634
:1034F000B1F00E943918688779878A879B87E091A5
:10350000BE05F091BF0584859585A685B785019692
:10351000A11DB11D84879587A687B787D9CFCDB761
:10352000DEB7E8E00C94F134A9E0B0E0EAE9FAE1B2
:103530000C94CB34E091BE05F091BF0542885388CE
:1035400064887588441555056605770518F080E090
:1035500090E0E2C019016A017B018D83209137025E
:10356000A0913502B0913602AD0160E070E04E836B
:103570005F836887798730E00E94A2344B015C0149
:10358000C301B2016C197D098E099F0969837A8391
:103590008B839C83C701B601A50194010E9453341B
:1035A00029013A01A5019401C301B2010E940F341F
:1035B000C61AD70AE80AF90AC701B6012E813F8167
:1035C000488559850E94533449015A012E813F8113
:1035D00048855985C501B4010E940F34C61AD70A1F
:1035E000E80AF90AC301B2010E94471AE091BE0538
:1035F000F091BF0560857185828593850E940717CC
:10360000680D791D8A1D9B1D0E94D51604EB14E0E0
:103610001F821E828E819F818215930509F44BC003
:103620008091350290913602A0E0B0E0C816D9062C
:10363000EA06FB06C0F17D817130E1F08FEF881A58
:10364000980AA80AB80A8091370290E0A0E0B0E09A
:1036500088169906AA06BB0698F09FEF491A590AE0
:10366000690A790AC301B2010E94471A812C912C80
:10367000540106C080E00E9495168823F9F267CFB6
:10368000E091BE05F091BF056085718582859385C7
:103690000E940717680D791D8A1D9B1D0E94D51673
:1036A000C12CD12C760149815A816B817C81452BBB
:1036B000462B472B21F45D81513061F526C0F60180
:1036C000EC54FD4F6D81613019F4D8018C9102C02A
:1036D0008081F801808349815A816B817C814150CE
:1036E00051096109710949835A836B837C836E8117
:1036F0007F816F5F7F4F7F836E837FEFC71AD70A0B
:10370000E70AF70A0F5F1F4F85CF80E00E949516EA
:1037100081111DCF8E819F812996E2E10C94E734BF
:10372000AAE1B0E0E6E9FBE10C94CB349C878B87FF
:10373000788F6F8BDC018D909D90AD90BC90BFEF2A
:103740008B1A9B0AAB0ABB0A8091100620903502A7
:103750003090360281FF11C0369427943694279416
:103760002FEF3FEF4FEF5FE02F83388749875A876E
:1037700044E050E05E834D830EC0369427948FEF73
:103780009FEFA0E0B0E08F839887A987BA87A2E077
:10379000B0E0BE83AD836101E12CF12CC501B40121
:1037A000A70196010E94533429013A01A70196010D
:1037B000C301B2010E940F3469837A838B839C8397
:1037C0008091270290912802A0912902B0912A02AB
:1037D000480E591E6A1E7B1E4091270250912802F6
:1037E0006091290270912A0280912B0290912C0203
:1037F000A0912D02B0912E02840F951FA61FB71F16
:10380000481659066A067B0608F0C4C0C301B20117
:103810000E94D516C501B401A70196010E94533438
:103820007A8F698F8090270290902802A0902902B9
:10383000B0902A0200912B0210912C0220912D02AF
:1038400030912E02800E911EA21EB31EA50194017E
:1038500021503109410951092D873E874F87588BE7
:10386000209123023091240240912502509126029A
:10387000298B3A8B4B8B5C8B80903702912CA12C3F
:10388000B12CAD81BE81A69FA001A79F500DB69F10
:10389000500D11245E8B4D8B00E010E0498D5A8D48
:1038A0004215530508F061C02D853E854F85588926
:1038B0004216530664067506E9F469897A898B898C
:1038C0009C89A50194010E945334CA01B901A70142
:1038D00096010E945334DC01CB010196A11DB11D5C
:1038E000E98DFA8DAF0160E070E084179507A607B7
:1038F000B707D8F1ED89FE89E00FF11FEC54FD4FB9
:1039000080819181A281B3812F81388549855A8533
:1039100082239323A423B5234D815E81040F151FB9
:10392000892B8A2B8B2BD1F4C980DA80EB80FC8029
:10393000898D9A8DC80ED91EE11CF11CAB85BC8502
:10394000CD92DD92ED92FC921397EF89F88D408233
:1039500051826282738280E090E01EC0298D3A8D90
:103960002F5F3F4F3A8F298F99CF89819A81AB8101
:10397000BC818C0D9D1DAE1DBF1D89839A83AB83B9
:10398000BC839FEF491A590A690A790A812C912C44
:10399000540122CF81E090E06A96E2E10C94E73492
:1039A000A9E1B0E0E6EDFCE10C94CB345C016A01E6
:1039B0007B0120911602309117024091180250911C
:1039C00019022E873F87488B598B0091100210E017
:1039D0000F5F1F4F0F7011270115110541F42F5F65
:1039E0003F4F4F4F5F4F2E873F87488B598B8091BA
:1039F000100681FD0DC08FEF9FEFA0E0B0E08A8B35
:103A00009B8BAC8BBD8BA2E0B0E0BD87AC870CC0BC
:103A10002FEF3FEF4FEF5FE02A8B3B8B4C8B5D8BA3
:103A200044E050E05D874C8719821A821B821C8219
:103A3000BE016B5F7F4FCE0101960E94901B892BC8
:103A400029F060E070E080E090E046C16E857F85FF
:103A5000888999890E94D51685E0000F111F8A95E3
:103A6000E1F7C8018C549D4F9A87898789819A8193
:103A7000AB81BC81E985FA85B58BA48B938F828F4E
:103A800048E050E0B501CF010E947D3743E050E0AF
:103A900062E272E089859A8508960E946E37A98550
:103AA000BA855C96CD92DD92ED92FC925F9780E2B2
:103AB0001B968C9380E00E9495168111C2CF89805D
:103AC0009A80AB80BC80C501B4010E9407176E8B41
:103AD0007F8B888F998F2090350230903602B0917D
:103AE0003702BB87910140E050E0C701B6010E9458
:103AF0005334EB854E2E512C612C712CCA01B90127
:103B0000A30192010E9453348901FB85F29D90012B
:103B1000F39D300D112440E050E0C701B6010E9432
:103B20005334672B682B692B11F401501109C10123
:103B30006C857D850E942B349B0140E050E0C501DF
:103B4000B4010E9453348091270290912802A091E1
:103B50002902B0912A02820F931FA41FB51F8D83E3
:103B60009E83AF83B887612C712C1B862C853D8585
:103B70001901412C512C80913502909136026C85AF
:103B80007D850E942B349B0140E050E069817A8161
:103B90008B819C810E9453349B01AC01C201B10115
:103BA0000E940F346B017C018D809E80AF80B884B1
:103BB000BE016B5F7F4FCE0101960E94901B892B47
:103BC00021F03B853F5F3B8783018D819E81AF81E3
:103BD000B88588169906AA06BB0621F0C501B4016E
:103BE0000E94D51680911006F601EC54FD4F601628
:103BF0007106A0F481FF0DC089819A81AB81BC81DF
:103C00002A893B894C895D8982239323A423B52388
:103C10000BC089819A81918380830FC081FF09C085
:103C20008A899B89AC89BD8980839183A283B38370
:103C300004C0AFEFBFEFB183A08380E00E94951670
:103C400080912B0290912C02A0912D02B0912E0216
:103C5000BC01CD01680D791D8A1D9B1D0E945D165A
:103C6000BFEF6B1A7B0A0615170508F084CFEB85AA
:103C7000EE2331F16E857F85888999890E94D5165A
:103C8000209137028091350290913602289FA00141
:103C9000299F500D1124C8010196489F9001499F0A
:103CA000300D589F300D1124C901A0E0B0E0E98526
:103CB000FA85848F958FA68FB78F81E00E94951625
:103CC00080911A0290911B0260E001960E948C186C
:103CD0006E897F89888D998D6996E2E10C94E7342D
:103CE000ABE0B0E0E6E7FEE10C94CD341B861A862B
:103CF000611571058105910521F460E070E0CB014B
:103D00007BC0409137022091350230913602429FAC
:103D1000F001439FF00D11248F0120E030E0980165
:103D200011270027061717072807390730F32B013B
:103D30003C01E091BE05F091BF058091160690917F
:103D40001706A0911806B091190684839583A6835F
:103D5000B78380E090E000E010E04E012AE0820EA0
:103D6000911C2AE1C22E22E0D22E34EBA32E34E0A5
:103D7000B32E7C012FEFE21AF20A60E00E948C1849
:103D80008823B1F09F928F92DF92CF92BF92AF9231
:103D90000E94AE378A859B850F900F900F900F90F1
:103DA0000F900F900817190708F48C01C701E1CF95
:103DB00081E0E816F10409F4A0CF0F5F1F4F003136
:103DC00027E2120708F099CF1F930F9381E192E049
:103DD0009F938F938E010F5F1F4F1F930F930E942E
:103DE0008C37B301A201C8010E94D01C0F900F9024
:103DF0000F900F900F900F902B96E0E10C94E93408
:103E0000FC01680F791F80E0E617F70739F0919100
:103E1000980F981708F49F5F892FF6CF0895209187
:103E2000C00025FFFCCF9093C5008093C40082E2C0
:103E30008093C00088E18093C10087E08093C20036
:103E40008091C00087FF03C08091C600F9CF08951C
:103E50009091C00095FFFCCF8093C60008950F930A
:103E60001F93CF93DF93EC018C01060F171FC01730
:103E7000D10721F089910E94281FF9CFDF91CF91BE
:103E80001F910F910895CF92DF92EF92FF92CF93FF
:103E9000DF939B01FC0152EFC52E59E4D52E52E071
:103EA000E52EF12C50E0A6B1A072B0E0A417B50742
:103EB00011F5A1E0CA1AD108E108F108F1F0A091CA
:103EC000C000A7FFF0CFA091C000D091C600A4FD14
:103ED00016C0CA2FC870A3FD14C02115310531F4D6
:103EE0000E94001FD81771F0C0E80CC0D083215089
:103EF00031093196D8CFC1E005C0C2E003C0C3E0AC
:103F000001C0C4E08C2FDF91CF91FF90EF90DF9044
:103F1000CF900895A1E0B0E0E0E9FFE10C94DB343C
:103F200040E20E94431F89838FE99FE00197F1F7E8
:103F300000C000008981882391F08EE40E94281F30
:103F400080910F028823B9F08EE40E949A0589813E
:103F5000805D8983CE0101960E9476260CC081E4A3
:103F60000E94281F80910F02882331F081E40E9473
:103F70009A0580E001C08FEF2196E2E00C94F734BF
:103F80000F931F93CF93DF93EC018B0180910F026E
:103F9000882351F0442321F085E40E949A050CC047
:103FA00083E40E949A050AC08FE79CE00197F1F72D
:103FB00000C00000442311F085E401C083E40E94A6
:103FC000281F8FE193E00197F1F700C00000B801CE
:103FD000CE010E942F1FB801CE010E94001F0E9437
:103FE000281FDF91CF911F910F9108954096FC01FA
:103FF000A591B4918C9184608C9380E090E00895B9
:1040000081E080932102809320027894E091400126
:10401000F09141010580F681E02D099580E090E066
:10402000089580912102813051F480911E02909177
:104030001F020A9790931F0280931E0204C01092E1
:104040000F021092200210922102E0914001F091A3
:1040500041010190F081E02D099580E090E0089504
:104060001092210280911E0290911F020A97909354
:104070001F0280931E0280912002882339F083E082
:10408000809321021092500110924F0180912102E1
:10409000E0914001F091410195E0899FE00DF11D13
:1040A00011240190F081E02D099580914F019091AC
:1040B0005001089582E080932102E0914001F09147
:1040C00041010284F385E02D099580E090E0089598
:1040D00080E090E00895FC0180911B0690911C0601
:1040E000893C910568F081E0809321027894E09109
:1040F0004001F09141010580F681E02D099508C04D
:10410000889748F07096A591B4918C9184608C93B7
:1041100080E090E008958FEF9FEF0895FC01828585
:10412000838781858287808581878EE28087148658
:104130000895EF92FF920F931F93CF93DF93809197
:104140001C0290911D02892B09F45AC060E08091F5
:104150001E0290911F020E948C18882309F4C6C089
:1041600060E270E08FE090E00E94672C20911C02DA
:1041700030911D0282E491E09F938F93C9010197D2
:10418000EAE0F0E0BF010E942B346F5F7F4F7F9326
:104190006F9380911E0290911F02BF010E942B34E9
:1041A0006F5F7F4F7F936F933F932F9389E692E0EA
:1041B0009F938F9384EB94E09F938F930E948C370F
:1041C00024EB34E040E050E06FEF7FEF81E00E94AD
:1041D000982C6DE270E08FE090E00E94672CC09117
:1041E0001E02D0911F028DB79EB70C960FB6F894A1
:1041F0009EBF0FBE8DBF87E0E82E85E0F82E44C03D
:1042000060E080911C0290911D020E948C1888230E
:1042100009F49CCF80911C0290911D02019690930D
:104220001D0280931C02ECCF60E0CE010E948C182E
:10423000882309F44DC08091B8052091BC0484FD09
:104240003AC086EE94E0FC013491231731F10396D5
:10425000E816F906C1F70DE71FEE203291F184EB65
:1042600094E00E948E2080914F019091500124EBA8
:1042700034E04AE852E5C817D90741F560EF7FEF0F
:1042800082E00E94982C219680911E0290911F023C
:104290000A96C817D90740F225C03196E4913091AB
:1042A000BD043E13D4CFFC013296E4913091BE049C
:1042B0003E13CDCF03C00FEF17E0CFCF00EE17E0D6
:1042C000CCCF2093BF041092C004CDCFB801D8CF7B
:1042D0002CE532E04AE852E560EE77E082E00E94A9
:1042E000702CD1CFD0931F02C0931E0280E090E0CB
:1042F000CDB7DEB7E6E00C94F33480911E029091C6
:104300001F028431910538F0449790931F028093E7
:104310001E020E94992080E090E0089510921F02F2
:1043200010921E020E94992080E090E008958091F2
:104330001C0290911D0201976AE070E00E942B34EC
:104340002AE0269FC001279F900D112490931F0201
:1043500080931E020E94992080E090E00895A5E0DD
:10436000B0E0E5EBF1E20C94CB3480E090E00E9409
:104370008529198204E110E024E130E03D832C839B
:104380008C809D803AE0830E911CAC80BD808AE0D9
:10439000A81AB1082FEF3FEFA801B401C5010E9490
:1043A0004A2A68019AE0C90ED11C78012AE0E21A73
:1043B000F1082FEF3FEFA601B7018C819D810E948C
:1043C000402A0E94C72D8111FCCF0E94C72D88234F
:1043D000E1F30E94332F60931B0670931C068093B9
:1043E0001D0690931E0620EE37E0A801B401C5011A
:1043F0000E944A2A20EE37E0A601B7018C819D81F8
:104400000E94402A60911B0670911C0680911D0637
:1044100090911E0639813230D1F0333019F13130AC
:1044200051F03B011C0180913B0190913C0144976C
:104430009D838C8324C02B01280E391E369427942B
:1044400000913D0110913E010451110918C0460E22
:10445000571E569447949B838A8324E130E03D8322
:104460002C830DC0660E771E769467942A813B815B
:10447000820F931F9C01369527953B832A833FEF3C
:1044800089E698E1315080409040E1F700C000009B
:1044900029812F5F2983243009F072CF0E94C72D14
:1044A0008111FCCF60913B0170913C0180E090E074
:1044B0000E9417366B017C01C201861997099D8302
:1044C0008C83BC01990F880B990B0E9419364B0104
:1044D0005C0120E030E040E252E4C701B6010E94F6
:1044E00002359B01AC01C501B4010E946F35A701E3
:1044F00096010E94A5360E94E1352C813D81621B08
:10450000730B77FF02C06F5F7F4F75956795661AD3
:10451000770A460E571E60913D0170913E0180E082
:1045200090E00E9417366B017C018A819B81821981
:1045300093099D838C83BC01990F880B990B0E9472
:1045400019364B015C0120E030E040E252E4C70143
:10455000B6010E9402359B01AC01C501B4010E9465
:104560006F35A70196010E94A5360E94E1352C8186
:104570003D81621B730B77FF02C06F5F7F4F7595A4
:104580006795261A370A8A819B81860F971F9B831E
:104590008A839F938F933F922F925F924F927F9245
:1045A0006F928DE392E09F938F9384EB94E09F93BF
:1045B0008F930E948C3760913D0170913E017695FA
:1045C000679524EBE22E24E0F22E00E010E02FEFBE
:1045D0003FEF41E084E190E00E94202C0FB6F89478
:1045E000DEBF0FBECDBF0E94C72D8823E1F3B3010C
:1045F0008DEB91E00E94A53DB20189EB91E00E9414
:10460000A53DB1018BEB91E00E94A53D6A817B81C4
:1046100087EB91E00E94A53D80E090E02596E2E1E5
:104620000C94E734A7E1B0E0E8E1F3E20C94CB347A
:104630001D8A80912102E0914001F091410195E0B5
:10464000899FE00DF11D112484819D89981708F040
:1046500082C0228133819D8984E1989FA001112429
:10466000DE01119680E090E0FA01E80FF91FE20FF9
:10467000F31FE491ED93019684319105A9F7E9893F
:10468000FA89E080E1FE63C0E2FE08C0EFE1F0E0FD
:10469000FC87EB8780EE9FEF988B8F874B845C8441
:1046A0008D809E80E985FA85FF8BEE8B6B807C8008
:1046B0002F803884260C371CAD84BE84E0FAEE24AB
:1046C000E0F89F01280D391D620101E0A101B4014C
:1046D000C3010E94562AC980DA802F853889C40117
:1046E00006976E897F8976956795680F791F7601A1
:1046F000820142E0C3010A960E94202CF6018081CB
:10470000843429F58181803311F12401F8E14F0EC1
:10471000511C310182E0681A710898E0890E911CE1
:10472000E2E12E1A31080DE015E09201A301B40177
:10473000C1010E94C02CF60183818C3341F400E05A
:1047400018EF9201A301B401C1010E94EF29FD8974
:10475000FF5FFD8B6ECF6796E2E10C94E7344096E5
:10476000FC01A591B4918C9182FB992790F99095C9
:1047700090FB82F98C938091B70582FB992790F981
:10478000909590FB82F98093B7050E94122380E0F8
:1047900090E008954096FC01A591B4918C9182FF20
:1047A00008C08091B70581608093B7058C918B7F9D
:1047B00009C08091B70580FF08C08E7F8093B70540
:1047C0008C9184608C930E94122380E090E0089585
:1047D0004096FC01A591B4918C9182FB992790F9A8
:1047E000909590FB82F98C930E94122380E090E0D8
:1047F0000895AF92BF92CF92DF92EF920F93CF9333
:10480000DF93CBE3D1E0488159814B505109A12C72
:10481000B12C8AE8C82E82E5D82EE12C01E028E1EF
:1048200031E068E270E08AE090E00E94562A488118
:1048300059814B50510999E5C92E9EECD92E00E0C3
:1048400028E131E068E270E08AE090E00E94562AB8
:10485000488159814C50510927E131E069E270E00B
:104860008BE090E00E94562A0E9412238FEF9FEF68
:104870009093500180934F010E949920DF91CF9136
:104880000F91EF90DF90CF90BF90AF900895AF92CF
:10489000BF92CF92DF92EF920F93CF9340913B0163
:1048A00050913C014B505109A12CB12C8AE8C82EE3
:1048B00082E5D82EE12C01E028E131E068E270E0E9
:1048C0008AE090E00E94562A40913B0150913C01C1
:1048D0004B50510999E5C92E9EECD92E00E028E1F4
:1048E00031E068E270E08AE090E00E94562A409150
:1048F0003B0150913C014C50510927E131E069E204
:1049000070E08BE090E00E94562A60914001709127
:10491000410140E050E020E030E080912102FB01C5
:1049200095E0899FE00DF11D1124848190E00297AC
:104930002817390750F50280F381E02DE40FF51FA9
:104940007096A591B491E0913F01F0E0022E02C073
:10495000F595E7950A94E2F78C91E0FB82F98C9348
:1049600090912102FB01C5E09C9FE00DF11D1124F7
:10497000E481F0E033972E173F0711F48B7F8C937F
:104980002F5F3F4F4C5E5F4FC8CF0E941223CF91E5
:104990000F91EF90DF90CF90BF90AF900895A0E07F
:1049A000B0E0E5EDF4E20C94D334CBE3D1E0488100
:1049B000598146505109A12CB12C8AE8C82E82E5B4
:1049C000D82EE12C01E025EF30E064E670E085E0D0
:1049D00090E00E94562A488159814650510999E534
:1049E000C92E9EECD92E00E025EF30E064E670E0A1
:1049F00085E090E00E94562A48815981475051092C
:104A000024EF30E065E670E086E090E00E94562AF0
:104A100024E3E22E22E0F22E0AE812E528E03CEF41
:104A200042E069E670E086E490E00E94FB2B68813A
:104A300079816850710928E03CEF4AE750E087E04F
:104A400090E00E944A2A0E941223CDB7DEB7EAE026
:104A50000C94EF34A0E0B0E0E0E3F5E20C94D33442
:104A6000EC01162F60911F067091200680913D0188
:104A700090913E0140978617970718F481E0809344
:104A800023069B01295F3F4F40913B0150913C0120
:104A90004B505109A12CB12C8BE7C82E85E2D82EA2
:104AA000E12C01E080912106909122060E94562A75
:104AB00060911F0670912006809121069091220638
:104AC0007E01112341F00BE715E22FEF3FEF41E0AC
:104AD0000E94FB2B07C00BE715E22FEF3FEF41E0F1
:104AE0000E94202C80911F0690912006089690939A
:104AF000200680931F06209123062223E1F02091B7
:104B00003D0130913E01285031092817390768F4DA
:104B100080912102843019F48AE090E002C08CE197
:104B200091E09093200680931F0680911F0690913C
:104B300020060E947929CDB7DEB7EAE00C94EF3465
:104B400061E00E942A250895A0E0B0E0EAEAF5E2DB
:104B50000C94D33484E190E0909322068093210654
:104B60008CE191E09093200680931F060E94CB2851
:104B700044E050E060E270E080911F0690912006D2
:104B80000E945F2980911F06909120060E9479293A
:104B90000E94C72880E090E00E94852986E0E82EE8
:104BA00082E0F82E00E010E028E03CEF42E06AE00E
:104BB00070E084E190E00E94FB2B9AEFE92E91E0F7
:104BC000F92E28E03CEF41E062E170E080EA90E0FD
:104BD0000E94FB2BCBE3D1E06881798128E03CEF98
:104BE0004EE150E080E090E00E944A2A0E941223A9
:104BF0002A813B8121503109488159814B5051090B
:104C0000A12CB12C6BE7C62E65E2D62EE12C01E07B
:104C100068E171E08AE090E00E94562A1092230633
:104C200060911F06709120068091210690912206C6
:104C30000E94672C87E095E00E94A02570E8E72E8F
:104C40000BE715E22FEF3FEF41E064E271E084E112
:104C500090E00E947C2BCDB7DEB7EAE00C94EF34F5
:104C6000EF920F931F938BE795E20E9485298AE0CC
:104C700090E09093220680932106909320068093E3
:104C80001F0646E050E060E371E00E945F298091DA
:104C90001F06909120060E947929109223066091A8
:104CA0001F067091200680912106909122060E9495
:104CB000672C87E095E00E94A02580E8E82E0BE7AE
:104CC00015E22FEF3FEF41E062E170E08AE090E013
:104CD0000E947C2B81E080930F0284E0809321026C
:104CE00080E090E01F910F91EF90089560E00E94A6
:104CF0002A250895A2E2B0E0E0E8F6E20C94D83468
:104D00008C01F62E82E28F1588F442E250E0B80161
:104D1000CE0101960E947D3760E0CE0101960E948F
:104D20002A258EEDF80E0E5D1F4FECCF60E0C80116
:104D30000E942A25A296E5E00C94F434A0E0B0E0AD
:104D4000E4EAF6E20C94D53480911D0690911E069B
:104D50008D9768E170E00E942B34C0911E02D091C3
:104D60001F022A97C60FD71F61E0CE010E948C1840
:104D70008091B80584FF67C0E091BE05F091BF0542
:104D8000C080D180E280F380C482D582E682F7823F
:104D90008091B4048E3209F03FC08091B5048E3208
:104DA000D9F5C114D104E104F10439F48FE290E0A3
:104DB000909343018093420137C060E080E090E02F
:104DC0000E948C18E091BE05F091BF058081918111
:104DD000A281B38184839583A683B78300E010E02A
:104DE00061E0C8010E948C18E091BE05F091BF05FA
:104DF00080819181A281B381C816D906EA06FB069B
:104E000029F4C482D582E682F78206C00F5F1F4F65
:104E10000F3F110529F7F5CF4CE050E064EB74E04B
:104E200082E491E00E947D3710921F0210921E02D0
:104E300010921D0210921C028FEF9FEF9093500171
:104E400080934F011CC0E4EBF4E001900020E9F7EF
:104E50003197BF01645B74406093240684EB94E057
:104E60000E947A26D0935001C0934F0180911E0278
:104E700090911F020A9790931F0280931E020E9436
:104E8000992061E0CE010E948C1880E090E0CDB7BF
:104E9000DEB7E8E00C94F134EF92FF920F931F938A
:104EA000CF930E944A2DC82F0E9400298EEA91E0DC
:104EB0000E94733D80933F0181700E942B290E94C4
:104EC00023299F938F9386E292E09F938F9384EBA5
:104ED00094E09F938F930E948C3784EBE82E84E0BC
:104EE000F82E00E010E02FEF3FEF42E062E271E0C9
:104EF00084E190E00E94202C0F900F900F900F9073
:104F00000F900F90CC2379F08DEB91E00E94813DC2
:104F1000019629F40E94C7280E94AF2104C00E9474
:104F2000C72D8111F7CFCF911F910F91FF90EF9077
:104F30000895FF920F931F93CF93DF93F0903F015B
:104F4000F0FAFF24F0F810923F0180912102A09125
:104F50004001B091410175E0879FA00DB11D112462
:104F600060E0262F30E014968C91149790E0FC01BD
:104F700032972E173F0714F51296ED91FC91139777
:104F800074E1679FE00DF11D112470960591149155
:104F9000E8010397281739077CF4888182FB4427AE
:104FA00040F950E0CA0101C0880F2A95EAF79091B4
:104FB0003F01892B80933F016F5FD3CF60913F0109
:104FC0008EEA91E00E94873D888182FD0EC080912B
:104FD0003F018170F81661F16FEF7FEF8DEB91E08B
:104FE0000E94A53D0E944C2723C0CCE3D2E006E9F5
:104FF00011E08EA580FF0EC04C8D5D8D6E8D7F8D76
:10500000C8010E94993D68A579A5C80104960E942F
:10501000A53D06C04FEF5FEFBA01C8010E94993D60
:1050200068960A5F1F4F82E0CC39D80711F7CFCFBF
:105030000E94112080E090E0CDB7DEB7E5E00C944F
:10504000F434A0E0B0E0E7E2F8E20C94D3340E943C
:10505000B92E362F272F60931B0670931C06809362
:105060001D0690931E0680912102A0914001B091EF
:10507000410195E0899FA00DB11D11241496AC90BB
:105080001497832F922F00911D0610911E0640E069
:1050900050E0B12CBA1451F112962D913C91139716
:1050A000240F351FF9013296C590D490F90134963A
:1050B000E590F490F9013696C591D491F9013896AE
:1050C00065917491C816D90668F4CC0DDD1D8C1756
:1050D0009D0740F4E016F10628F46E0D7F1D0617BB
:1050E000170738F0B3944C5E5F4FD4CF80E090E068
:1050F00001C0C901CDB7DEB7EAE00C94EF3484B14A
:10510000836084B98AB18C6F8AB987B18F6187B99E
:1051100088B18B6088B98FE39CE90197F1F700C0F3
:105120000000089544988FE59AEE0197F1F700C0CA
:105130000000449A8FE59AEE0197F1F700C0000055
:1051400008959BB19370282F2C7F922B9BB995B11A
:105150009C7F8370892B85B94198419A0895409826
:105160002FEF89EF90E0215080409040E1F700C0A0
:10517000000029B193B1409A2C7F892F8370822B34
:105180000895429843980E94A128439A089589E27D
:105190000E94C128089588E20E94C1280895CF93F3
:1051A000C82F429A4398892F0E94A1288C2F0E94D1
:1051B000A128439ACF910895CF9384B18C7F84B96D
:1051C0008AB183708AB9429A43980E94AF28C82F47
:1051D0000E94AF28439A94B1936094B99AB19C6F9E
:1051E0009AB92C2F30E0322F2227A901482BCA016F
:1051F000CF910895429A43980E94A128439A089516
:105200000E947F280E9492282FEF83EC99E0215082
:1052100080409040E1F700C0000081E20E94C12878
:105220008AE30E94C12885E50E94FA2881E10E9454
:10523000C1282FEF81EE94E0215080409040E1F7AB
:1052400000C00000089583ED0E94C1280E94DC2860
:105250000E94DC280895CF93C82F86E30E94C128BE
:10526000CC2321F0C13029F488E901C088E40E94F0
:10527000FA28CF910895A0E0B0E0E1E4F9E20C94BF
:10528000D5346C018B017A01E9018AE20E94C128C0
:10529000C6010E94CF28C7010E94CF288BE20E943E
:1052A000C128C8010E94CF28CE010E94CF288CE2DD
:1052B0000E94C128CDB7DEB7E8E00C94F134EF923C
:1052C000FF920F931F93CF93DF937C018B01EA0131
:1052D00083E30E94C128C7010E94CF28C8010E9411
:1052E000CF28CE010E94CF28CDB7DEB7E6E00C94E0
:1052F000F334CF93DF93EC0187E30E94C128CE0102
:105300000E94CF28DF91CF910895CF92DF92EF9244
:10531000FF92CF93DF93EC01209151013091520124
:10532000215031094091530150915401415051098C
:1053300060E070E080E090E00E943B29C12C8CE2AC
:10534000D82EEE24E394F12CCE010E94CF2881E0E8
:10535000C81AD108E108F108B9F7DF91CF91FF90A1
:10536000EF90DF90CF900895CF92DF92EF92FF926F
:105370000F931F93DA01A81BB90B1196F901E61BD5
:10538000F70B3196AE9F6001AF9FD00CBE9FD00C43
:105390001124E12CF12C0E943B29C114D104E10419
:1053A000F10449F0C8010E94CF2881E0C81AD10851
:1053B000E108F108F2CF1F910F91FF90EF90DF907D
:1053C000CF900895CF93DF93EA019B01AC010E9437
:1053D0003B29CE010E94CF28DF91CF910895A0E014
:1053E000B0E0E5EFF9E20C94CD347C01EB013A0139
:1053F00029016A01C81AD90A5901A61AB70ACC0CA0
:10540000DD1CAA0CBB1CA8010E94E229AC14BD043F
:10541000C8F4C601969587954501881A990AE6143D
:10542000F70449F197FC03C021968C189D088FEF73
:10543000E81AF80A8A0C9B1CA801BE01C7010E9449
:10544000E229EDCFC501969587954601881A990AFC
:10545000C415D50581F097FC05C08FEFE81AF80A4E
:105460008A189B0821968C0C9D1CA801BE01C701BF
:105470000E94E229EDCFCDB7DEB7E0E10C94E9342C
:105480000F931F9389019A01AC010E94B4291F91C7
:105490000F9108950F931F93FB01BA0189019A019F
:1054A000AF010E94B4291F910F9108954F925F920E
:1054B0006F927F928F929F92AF92BF92CF92DF9224
:1054C000EF920F931F93CF93DF933C014B01EA01BF
:1054D0002901013021F486010E94B42916C09601E9
:1054E000A2010E94402A9601A201B401CE010E94AD
:1054F000402A9601A401BE01C3010E944A2A9601D6
:10550000A201BE01C3010E944A2AEE20A1F0A5011A
:10551000B401C3010E94E229A501B201C3010E94A6
:10552000E229A501B401CE010E94E229A501B20140
:10553000CE010E94E229DF91CF911F910F91EF9050
:10554000DF90CF90BF90AF909F908F907F906F90A3
:105550005F904F900895ADE0B0E0E1EBFAE20C947B
:10556000CB347C013B015D874C872B8781E090E049
:105570009C01241B350B3A83298317014B017C8343
:105580006B83270143E050E058874F839E838D83D0
:105590002D813E81215031093A872987CC84DD84D1
:1055A000C60CD71C3B85313039F59801A601B101F5
:1055B000C2010E944A2A9801A3018C859D85481B3F
:1055C000590BB101C2010E944A2A98014B815C81AA
:1055D000AC84BD84AE0CBF1CB50167018C859D8574
:1055E000C81AD90AC6010E944A2A9801A401B50125
:1055F000C6010E944A2A38C0A801B601C1010E9412
:10560000E229A8016B817C81AC84BD84AE0CBF1CF7
:10561000C5010E94E229A801B601C2010E94E22947
:10562000A8016B817C8167012C853D85C21AD30A54
:10563000C6010E94E229A801B401C5010E94E22925
:10564000A80153018C859D85A81AB90AB501C1012D
:105650000E94E229A801B501C2010E94E229A80125
:10566000B401C6010E94E22929813A8137FF0BC0AB
:105670002D813E8149815A818F819885480F591F1C
:105680005A83498316C02D813E8189859A854C8530
:105690005D85841B950B880F991F059649815A815A
:1056A000480F591F5A8349838C859D8501979D8793
:1056B0008C874D815E814F5F5F4F5E834D838F810D
:1056C0009885029698878F8391E0491A51084FEF89
:1056D000241A340A8B819C8101969C838B8391E0F0
:1056E000891A91084C855D85421753070CF050CFFD
:1056F0002D96E2E10C94E7342F923F924F925F9205
:105700007F928F929F92AF92BF92CF92DF92EF9251
:10571000FF920F931F93CF93DF93FC01542E490107
:10572000411102C055245394852D90E09C018E17A1
:105730009F0708F4CF0143E0220F331F4A95E1F79A
:10574000AB0141505109240F351FAC0141505109A3
:10575000E5E05E9E400D511D11240E943B2985E02D
:10576000E89E70011124C12CD12CE0EAEE1AF10858
:1057700022242394312C0C2C02C0220C331C0A94BA
:10578000E2F7712CA12CB12CF701EA0DFB1DE25FB1
:10579000F84FC491D0E0C221D321412C209711F0C1
:1057A000C40101C0C8010E94CF2843945410F6CF11
:1057B0008FEFA81AB80AE5E0AE16B10429F7739482
:1057C0005710E0CF8FEFC81AD80AE8E0CE16D10400
:1057D00079F6DF91CF911F910F91FF90EF90DF90BD
:1057E000CF90BF90AF909F908F907F905F904F90A1
:1057F0003F902F900895A0E0B0E0E1E0FCE20C942F
:10580000CC346C015B01342E4901380186E0489F9D
:1058100020011124F701E490EF012196EE2059F0C8
:1058200083019401432DB501C6010E947C2BC40C59
:10583000D51CFE01F0CFCDB7DEB7E1E10C94E83422
:10584000A0E0B0E0E6E2FCE20C94CC343C016B0159
:10585000342E5901480186E0489F20011124E701B8
:10586000E99084019501432DB601C3010E947C2B70
:10587000640C751C88818052803690F3CDB7DEB7FA
:10588000E1E10C94E834A0E0B0E0E9E4FCE20C943F
:10589000CB34EC015B01D42E4901380186E0489FEE
:1058A000100111242701F201E1902F0183019401DD
:1058B0004D2DB501CE010E947C2BC20DD31DCA9483
:1058C000C110F1CFCDB7DEB7E2E10C94E73490938D
:1058D0002806809327067093260660932506089570
:1058E000EF92FF920F931F93CF93C82F80912506BD
:1058F0009091260679018A019B014C2FBC01809171
:105900002706909128060E94FB2B809125069091F6
:1059100026062CE0C29F800D911D1124909326062F
:1059200080932506CF911F910F91FF90EF900895DE
:10593000EF92FF920F931F93CF93C82F809125066C
:105940009091260679018A019B014C2FBC01809120
:105950002706909128060E94202C80912506909180
:1059600026062CE0C29F800D911D112490932606DF
:1059700080932506CF911F910F91FF90EF9008958E
:10598000A0E0B0E0E6ECFCE20C94D134FC01EB01C9
:105990005901261B370BDA01A81BB90B0E949A3458
:1059A0006B017C0195012150310941505109BE0123
:1059B000CF010E943B29E801812C912C54018C14C9
:1059C0009D04AE04BF0461F0FE01859194910E9494
:1059D000CF288FEF881A980AA80AB80A2296EFCF24
:1059E000CDB7DEB7ECE00C94ED34E0912E06F091EB
:1059F0002F0681E090E09C0100902B0602C0220F50
:105A0000331F0A94E2F7322F3095418134233183DA
:105A1000E0912E06F0912F063281232B228338B19C
:105A2000AC010090300602C0440F551F0A94E2F703
:105A3000242F2095232328B937B1AC0100902906E3
:105A400002C0440F551F0A94E2F7242F2095232308
:105A500027B938B1AC010090290602C0440F551F88
:105A60000A94E2F7242F2095232328B9E0912C06ED
:105A7000F0912D0600902A0602C0880F991F0A9403
:105A8000E2F7809592818923828385E38A95F1F7F5
:105A90000000089587E880937A0086EB91E00E94E9
:105AA000733D8F3F31F18093290685EB91E00E9491
:105AB000733D80932B0682EB91E00E94733D8093AF
:105AC0002A068FEA91E00E94733D8093300683EBB3
:105AD00091E00E94813D90932F0680932E0680EBEB
:105AE00091E00E94813D90932D0680932C0681E0E9
:105AF000089580E0089548B181E090E09C01009015
:105B0000290602C0220F331F0A94E2F7242B28B97A
:105B100048B19C010090300602C0220F331F0A9446
:105B2000E2F7242B28B9E0912E06F0912F069C0174
:105B300000902B0602C0220F331F0A94E2F7318136
:105B4000232B218347B19C010090300602C0220F15
:105B5000331F0A94E2F7242B27B947B19C01009028
:105B6000290602C0220F331F0A94E2F7242B27B91B
:105B7000E0912C06F0912D0600902A0602C0880FB5
:105B8000991F0A94E2F79181892B81830895CF931D
:105B9000DF93F8940E94F52CE0912E06F0912F06E9
:105BA000C081D0E000902B0602C0D595C7950A941D
:105BB000E2F7C170DD2781E0C8270E947B2D789431
:105BC0008C2FDF91CF910895E0912E06F0912F0652
:105BD00020912B0640913006882309F45BC081E0B8
:105BE00090E0BC0102C0660F771F2A95E2F79B0187
:105BF0002095318132233183E0912E06F0912F06DA
:105C000032812323228357B19C0101C0220F4A9580
:105C1000EAF7252B27B938B1AC010090300602C055
:105C2000440F551F0A94E2F7242F2095232328B907
:105C300037B1AC010090290602C0440F551F0A94E9
:105C4000E2F7242F2095232327B938B1AC01009027
:105C5000290602C0440F551F0A94E2F7242F20950D
:105C6000232328B9E0912C06F0912D0600902A06F6
:105C700002C0880F991F0A94E2F79181982B9183B3
:105C8000E0912C06F0912D069281892B82838091E0
:105C900029065AC081E090E0BC0102C0660F771F60
:105CA0002A95E2F79B013181322B3183E0912E0658
:105CB000F0912F06209532812323228337B1BC0136
:105CC00002C0660F771F4A95E2F7262F20952323FF
:105CD00027B938B1AC010090300602C0440F551FFF
:105CE0000A94E2F7242F2095232328B947B19C0179
:105CF0000090290602C0220F331F0A94E2F7242BDA
:105D000027B948B19C010090290602C0220F331F19
:105D10000A94E2F7242B28B9E0912C06F0912D0685
:105D200000902A0602C0880F991F0A94E2F7809516
:105D3000918198239183E0912C06F0912D06928118
:105D40008923828380913006806480937C0072E096
:105D50007A95F1F700C080917A00806480937A0090
:105D600080917A0086FDFCCF809178009091790037
:105D70000895A8E0B0E0EFEBFEE20C94CB34F89489
:105D80004090530150905401612C712C89EB91E0AB
:105D90000E94813D8C018DEB91E00E94813D6C0160
:105DA000E12CF12C80E00E94E42D98878F83809075
:105DB000510190905201940140E050E029833A83D0
:105DC0004B835C8387EB91E00E94813D9E838D83B2
:105DD0008BEB91E00E94813D4C01A12CB12C81E024
:105DE0000E94E42D1C010E947B2D78944F815885E0
:105DF000CA01A0E0B0E09C01AD012C193D094E099B
:105E00005F09C301B2010E940F3420E030E0A90114
:105E100098012C193D094E095F090E9475346901EA
:105E2000C101A0E0B0E09C01AD01281939094A097F
:105E30005B0969817A818B819C810E940F34AD81DD
:105E4000BE818D0120E030E0A901980128193909AF
:105E50004A095B090E9475347901C701B601289689
:105E6000E2E10C94E7340F931F93CF93DF93F89400
:105E700080E00E94E42D8C0181E00E94E42DEC0181
:105E80000E947B2D7894B801CE01DF91CF911F91B4
:105E90000F910895CF92DF92EF92FF92CF93DF930D
:105EA00020E330E040E050E0BA0180E00E94941A24
:105EB0008091B404813409F05EC08091B5048435CA
:105EC00009F059C08091B604883309F054C080911C
:105ED000B704883509F04FC08091B8049091B90497
:105EE000019709F048C08091BA049091BB040197D2
:105EF00009F041C08091C604813011F092E101C0E7
:105F00009AE190933506823019F080E890E002C063
:105F100080E091E09093340680933306C090D004E3
:105F2000D090D104E090D204F090D304C7E3D6E03F
:105F300020E230E0B701A60180E00E94941A892B8C
:105F400029F4809133069091340617C0C992D992F2
:105F5000E992F9928091B4049091B504A091B604AD
:105F6000B091B704C80ED91EEA1EFB1E86E0CF3DD5
:105F7000D807F1F6E6CF80E090E0DF91CF91FF9077
:105F8000EF90DF90CF900895A0E1B0E0EAECFFE25F
:105F90000C94CB34FB01588B4F87019798878F83E4
:105FA00080913506282F30E03A8729878F819885A0
:105FB000B9010E942B3401E0060F80E1AF85B8895A
:105FC0008C938091330690913406918380830E9454
:105FD000F631EFE4F2E33197F1F700C00000809171
:105FE0003606081761F1E02EE81AE7FCE194C12CAF
:105FF000D12C0E2C000CFF08CE14DF0498F40E9464
:10600000F631882329F087EE91EC0197F1F704C06F
:10601000AFECB2E51197F1F700C00000BFEFCB1A6B
:10602000DB0AEACF0E94F631882349F0EFEFF3EF65
:1060300021E0E150F0402040E1F700C00000009373
:1060400036060E94EF316C0110E001501109A801E1
:10605000440F551F440F551F5E834D83FA01E95CC1
:10606000F94F80809180A280B38081149104A104B3
:10607000B10419F4E12CF12C92C120E230E0B50119
:10608000A40180E00E94941A8091BC0490E008175B
:10609000190781F72090BE043090BF042114310409
:1060A00049F38091C8049091C904A091CA04B091A9
:1060B000CB04880E991EAA1EBB1E28E030E0B50155
:1060C000A40180E00E94941A8091B4049091B504D8
:1060D000A091B604B091B704880E991EAA1EBB1EEB
:1060E000C10123E0880F991F2A95E1F7A5019401CA
:1060F000281B390B410951092B873C874D875E8747
:1061000034E03C8300E010E01B82812C912C540190
:10611000E12CF12C4B845C846D847E841A8219827C
:1061200028E030E0B301A20180E00E94941A892B9C
:1061300009F44EC02091B50424FD45C08F81988597
:1061400069857A850E942B348F5F9091B4048913FE
:106150003AC08091B6049091B704AC014C195D0926
:106160000115110571F0141615061CF417FD09C070
:1061700005C04115510539F117FF25C040175107DA
:1061800014F5909332068093310622FD04C0AF854A
:10619000B8892C9305C0822F8260EF85F8898083AF
:1061A000AF85B8898C9186FF03C0BB81BF5FBB837D
:1061B0008090B8049090B904A090BA04B090BB0449
:1061C0008A01E980FA80E8E04E0E511C611C711CC6
:1061D00029813A812F5F3F4F3A8329832216330664
:1061E00009F09ECFAF85B8898C91811114C0809140
:1061F0003106909132069093B5058093B405EF85F2
:10620000F88980818F7789838083FB81F11115C0A4
:106210000FEF1FEF54C00E94EF319C0186549A4942
:106220008B3B45E6940708F0C9010E94D9315C8197
:1062300051505C8351116ECFDACFED81FE81E95C64
:10624000F94F40805180628073808091C8049091A2
:10625000C904A091CA04B091CB04480E591E6A1E0D
:106260007B1E0FEF1FEF28E030E0B301A20180E0BA
:106270000E94941A4091B4045091B5046091B60400
:106280007091B704411551056105710599F0809130
:10629000B90490E0E816F90641F48091B804803121
:1062A00021F40091BA041091BB04440E551E661EE1
:1062B000771ED9CFAF85B8898C918F7B8C93811451
:1062C0009104A104B104A1F0209133063091340669
:1062D000ED81FE81E95CF94F4081518162817381DA
:1062E000480D591D6A1D7B1D80E00E94941A7C0197
:1062F0008981882311F0E12CF12C17FF0AC08091CD
:10630000310690913206C816D906E0F086549A49B3
:1063100019C0D801AC54BB4F5D0100E011E02091E1
:10632000330630913406C501845B9440821793078D
:1063300030F70E945E37B8010E943F34F501819327
:106340005F01EDCF9C012C193D098AEB95E6B10167
:106350000E942B34C20ED31EFBEBCF16F5E6DF06F0
:1063600020F02AEBC21A25E6D20ACB018C0D9D1D26
:106370008B3B35E6930710F08A5B95460E94D93136
:106380000E94F631882329F08FE39FE10197F1F70E
:1063900004C0AFE3BFE11197F1F700C00000EF8543
:1063A000F889808180958083C7016096E2E10C9432
:1063B000E734209184003091850036952795821727
:1063C000930718F4B19AB19BFECF209184003091CD
:1063D00085003695279528173907B8F308958091D9
:1063E00084009091850096958795089580913F014E
:1063F00083FB882780F908952091E1063091E20619
:106400003695279540E050E060E472E48FE090E03C
:106410000E945334C90101970E940F1F08958F9263
:106420009F92AF92BF92EF92FF920F931F93CF93E1
:10643000DF93EC014C01A12CB12CE091BE05F09151
:10644000BF05428953896489758984169506A60615
:10645000B70608F05CC0415051096109710997E025
:1064600076956795579547959A95D1F74F5F5F4F0A
:106470006F4F7F4F7F936F935F934F93CE01880F42
:10648000892F881F990B919501969F938F9387E28F
:1064900099E09F938F9384EB94E09F938F930E9456
:1064A0008C3734EBE32E34E0F32E0AE812E520EECD
:1064B0003FEF42E064E870E083E290E00E94202C2D
:1064C00020E830E0B501A40180E00E94941AE4E3E2
:1064D000F5E02DB73EB7265F3F4F0FB6F8943EBFAD
:1064E0000FBE2DBF34E0E43BF30719F09291938384
:1064F000F9CF87FD06C09AEF9093B60480933605D6
:1065000003C09CEF9093B604C80FD11D18C081E260
:10651000E82E89E0F82E0AE812E520EE3FEF42E08F
:1065200064E870E083E290E00E94FB2B83E890E057
:106530000E9491058EEF8093B604C0E0D0E085E51F
:106540008093B4048093B50463E870E084EB94E036
:106550000E942F1F63E870E084EB94E00E94001F0C
:106560000E94281F8FEF95EA2EE081509040204036
:10657000E1F700C00000CE01DF91CF911F910F9194
:10658000FF90EF90BF90AF909F908F90089528E07C
:1065900030E040E050E0BA0180E00E94941A90910F
:1065A000B4048091B705963471F49091B504953593
:1065B00051F49091B6049A3431F49091B70499341F
:1065C00011F4826001C08D7F8093B7058091B7057B
:1065D00082FF03C088EE93E002C088E592E09093CA
:1065E000E2068093E1060E94FC311092E0061092D0
:1065F000DF060895A0E0B0E0E0E0F3E30C94CF34D0
:106600006C014601A12CB12CE091BE05F091BF05B3
:1066100082899389A489B58988169906AA06BB063A
:1066200008F045C028E030E0B501A40180E00E94F8
:10663000941AC091B804D091B9048091B4048436FE
:10664000B1F48091B504813671F58091B604843738
:1066500051F58091B704813631F58091DF06909134
:10666000E00601969093E0068093DF0620C0823614
:10667000D1F48091B5048136B1F48091B6048537A8
:1066800091F48091B704843671F48091B70582FD4E
:10669000B8CF8091BA049091BB049093E2068093A6
:1066A000E1060E94FC312896CC0EDD1EAACF84EBB9
:1066B00094E06090BA047090BB04C091B804D0918B
:1066C000B9047F926F92DF93CF932091E2062F93CC
:1066D0002091E1062F9321E039E03F932F939F9380
:1066E0008F930E948C3794EBE92E94E0F92E0AE800
:1066F00012E520EE37E041E069E970E08FE090E0DC
:106700000E94202C8DB79EB70A960FB6F8949EBFB4
:106710000FBE8DBFC301009741F0EFE9FFE0319755
:10672000F1F700C000000197F6CFE091BE05F091AF
:10673000BF0582899389A489B58988169906AA0616
:10674000BB0608F064C08091E0068F938091DF065D
:106750008F9383EF98E09F938F9384EB94E09F93C4
:106760008F930E948C3784EBE82E84E0F82E0AE8A1
:1067700012E520EE3FEF42E064E870E083E290E053
:106780000E94202C8601085F1F4F0F900F900F90E2
:106790000F900F900F90DD24D39480E091E020972C
:1067A00031F1C130F1E0DF0720F05E01BA94EC0175
:1067B00002C0A12CB12CA80160E070E09E0180E035
:1067C0000E94941A080F191FBE0184EB94E00E94E6
:1067D0002F1FDD2041F08091B6048E3F21F41092EE
:1067E000E0061092DF06D12CCE01E501D8CF8091D2
:1067F000DF069091E006892B61F48FEF93ECE9E0DE
:1068000081509040E040E1F700C0000002C000E08D
:1068100010E0C801CDB7DEB7EEE00C94EB34DB013D
:106820008F939F930E94B834BF91AF91A29F800D28
:10683000911DA39F900DB29F900D11240895991B57
:1068400079E004C0991F961708F0961B881F7A9567
:10685000C9F780950895AA1BBB1B51E107C0AA1F69
:10686000BB1FA617B70710F0A61BB70B881F991FF1
:106870005A95A9F780959095BC01CD01089597FB95
:10688000072E16F4009407D077FD09D00E942B3410
:1068900007FC05D03EF4909581959F4F0895709523
:1068A00061957F4F0895A1E21A2EAA1BBB1BFD0123
:1068B0000DC0AA1FBB1FEE1FFF1FA217B307E407DF
:1068C000F50720F0A21BB30BE40BF50B661F771F37
:1068D000881F991F1A9469F7609570958095909517
:1068E0009B01AC01BD01CF010895052E97FB1EF45D
:1068F00000940E948C3457FD07D00E94533407FC4B
:1069000003D04EF40C948C345095409530952195DD
:106910003F4F4F4F5F4F08959095809570956195CB
:106920007F4F8F4F9F4F0895EE0FFF1F0590F491FB
:10693000E02D09940E94A234332312F48A1B9B0B8E
:106940000C94B334A29FB001B39FC001A39F700DFC
:10695000811D1124911DB29F700D811D1124911D67
:1069600008950E94A234B7FF0895821B930B0895E7
:106970000E94A234A59F900DB49F900DA49F800DFE
:10698000911D11240895B7FF0C94B8340E94B834B7
:10699000821B930B08952F923F924F925F926F92BA
:1069A0007F928F929F92AF92BF92CF92DF92EF929F
:1069B000FF920F931F93CF93DF93CDB7DEB7CA1B20
:1069C000DB0B0FB6F894DEBF0FBECDBF09942A884B
:1069D000398848885F846E847D848C849B84AA84F3
:1069E000B984C884DF80EE80FD800C811B81AA8180
:1069F000B981CE0FD11D0FB6F894DEBF0FBECDBF4B
:106A0000ED0108955058BB27AA270E941A350C940F
:106A10006B360E945D3638F00E94643620F039F4FF
:106A20009F3F19F426F40C945A360EF4E095E7FBD8
:106A30000C945436E92F0E947C3658F3BA1762073B
:106A400073078407950720F079F4A6F50C949E3619
:106A50000EF4E0950B2EBA2FA02D0B01B901900179
:106A60000C01CA01A0011124FF27591B99F0593FBD
:106A700050F4503E68F11A16F040A22F232F342F05
:106A80004427585FF3CF469537952795A795F04053
:106A90005395C9F77EF41F16BA0B620B730B840B68
:106AA000BAF09150A1F0FF0FBB1F661F771F881F20
:106AB000C2F70EC0BA0F621F731F841F48F4879578
:106AC00077956795B795F7959E3F08F0B0CF93956A
:106AD000880F08F09927EE0F9795879508950E94E3
:106AE00083350C946B360E94643658F00E945D36F4
:106AF00040F029F45F3F29F00C94543651110C9466
:106B00009F360C945A360E947C3668F39923B1F371
:106B1000552391F3951B550BBB27AA2762177307C3
:106B2000840738F09F5F5F4F220F331F441FAA1F57
:106B3000A9F335D00E2E3AF0E0E832D09150504013
:106B4000E695001CCAF72BD0FE2F29D0660F771FC1
:106B5000881FBB1F261737074807AB07B0E809F0A7
:106B6000BB0B802DBF01FF2793585F4F3AF09E3F2C
:106B7000510578F00C9454360C949F365F3FE4F343
:106B8000983ED4F3869577956795B795F7959F5F6F
:106B9000C9F7880F911D9695879597F90895E1E0BB
:106BA000660F771F881FBB1F621773078407BA071A
:106BB00020F0621B730B840BBA0BEE1F88F7E09575
:106BC00008950E94E8356894B1110C949F36089599
:106BD0000E94843688F09F5798F0B92F9927B751B3
:106BE000B0F0E1F0660F771F881F991F1AF0BA9571
:106BF000C9F714C0B13091F00E949E36B1E00895FB
:106C00000C949E36672F782F8827B85F39F0B93FEC
:106C1000CCF3869577956795B395D9F73EF4909523
:106C20008095709561957F4F8F4F9F4F0895E894A1
:106C300009C097FB3EF490958095709561957F4FC4
:106C40008F4F9F4F9923A9F0F92F96E9BB27939572
:106C5000F695879577956795B795F111F8CFFAF482
:106C6000BB0F11F460FF1BC06F5F7F4F8F4F9F4FB3
:106C700016C0882311F096E911C0772321F09EE811
:106C8000872F762F05C0662371F096E8862F70E077
:106C900060E02AF09A95660F771F881FDAF7880F51
:106CA0009695879597F9089597F99F6780E870E022
:106CB00060E008959FEF80EC089500240A94161672
:106CC000170618060906089500240A9412161306DA
:106CD000140605060895092E0394000C11F4882368
:106CE00052F0BB0F40F4BF2B11F460FF04C06F5F84
:106CF0007F4F8F4F9F4F089557FD9058440F551F5A
:106D000059F05F3F71F04795880F97FB991F61F02D
:106D10009F3F79F087950895121613061406551FA4
:106D2000F2CF4695F1DF08C0161617061806991F10
:106D3000F1CF86957105610508940895E894BB2705
:106D400066277727CB0197F908950E94B8360C94EF
:106D50006B360E945D3638F00E94643620F0952331
:106D600011F00C9454360C945A3611240C949F361E
:106D70000E947C3670F3959FC1F3950F50E0551F2C
:106D8000629FF001729FBB27F00DB11D639FAA2780
:106D9000F00DB11DAA1F649F6627B00DA11D661FCF
:106DA000829F2227B00DA11D621F739FB00DA11DF0
:106DB000621F839FA00D611D221F749F3327A00DAA
:106DC000611D231F849F600D211D822F762F6A2F46
:106DD00011249F5750409AF0F1F088234AF0EE0FAB
:106DE000FF1FBB1F661F771F881F91505040A9F7D8
:106DF0009E3F510580F00C9454360C949F365F3FB3
:106E0000E4F3983ED4F3869577956795B795F79513
:106E1000E7959F5FC1F7FE2B880F911D969587958B
:106E200097F908958F929F92AF92BF92CF92DF927F
:106E3000EF92FF92CF93DF93EC01688179818A8191
:106E40009B81611571058105910521F464E279ED5D
:106E50008BE597E02DE133EF41E050E00E9475347F
:106E600049015A019B01AC01A7EAB1E40E94B83480
:106E70006B017C01ACEEB4EFA50194010E94C63415
:106E8000DC01CB018C0D9D1DAE1DBF1DB7FF03C0E6
:106E90000197A109B04888839983AA83BB839F7710
:106EA000DF91CF91FF90EF90DF90CF90BF90AF90A8
:106EB0009F908F9008950E941237089585E591E084
:106EC0000E9412370895A0E0B0E08093550190939E
:106ED0005601A0935701B09358010895FB01DC01BE
:106EE0004150504048F005900D920020C9F701C074
:106EF0001D9241505040E0F70895FB01DC014150E4
:106F0000504048F001900D920020C9F701C01D9239
:106F100041505040E0F70895AEE0B0E0E2E9F7E319
:106F20000C94D9340D891E898EE08C831A830983D1
:106F30008FEF9FE79E838D83AE01475E5F4F6F8922
:106F4000788DCE0101960E94C737EF81F885E00F5A
:106F5000F11F10822E96E4E00C94F534AEE0B0E020
:106F6000E4EBF7E30C94DB348DE08C838B899C8914
:106F70009A838983AE01495E5F4F6D897E89CE0118
:106F800001960E94443B2E96E2E00C94F734ABE06D
:106F9000B0E0EDECF7E30C94CB346C017B018A019B
:106FA000FC0117821682838181FFCCC1CE0101963C
:106FB0003C01F6019381F70193FD859193FF819147
:106FC0007F01882309F4BAC1853239F493FD859194
:106FD00093FF81917F01853229F4B60190E00E94F0
:106FE000BD3CE7CF912C212C312CFFE1F315D8F0DB
:106FF0008B3279F038F4803279F08332A1F4232D8A
:1070000020611DC08D3261F0803369F4232D216031
:1070100016C0832D8260382EE32DE4603E2E2AC0F8
:10702000F32DF8601DC037FC2DC020ED280F2A304D
:1070300040F08E32B9F436FC81C1232D2064322E0B
:1070400019C036FE06C08AE0989E200D1124922EAB
:1070500011C0EAE02E9E200D1124222EF32DF062A5
:107060003F2E08C08C3621F4832D8068382E02C054
:10707000883641F4F70193FD859193FF81917F015B
:107080008111B3CF982F9F7D9554933028F40C5FD6
:107090001F4F9FE399830DC0833631F0833771F022
:1070A000833509F059C021C0F801808189830E5FC2
:1070B0001F4F88248394912C530113C02801F2E0C0
:1070C0004F0E511CF801A080B18036FE03C0692D1F
:1070D00070E002C06FEF7FEFC5010E94743C4C016D
:1070E0008201F32DFF773F2E16C0280122E0420EC9
:1070F000511CF801A080B18036FE03C0692D70E0FC
:1071000002C06FEF7FEFC5010E94693C4C01F32D77
:10711000F0683F2E820133FC1BC0822D90E0881660
:107120009906B0F4B60180E290E00E94BD3C2A943A
:10713000F4CFF50137FC859137FE81915F01B601EF
:1071400090E00E94BD3C21102A9421E0821A91080F
:107150008114910471F7E8C0843611F0893641F545
:10716000F80137FE07C060817181828193810C5FD5
:107170001F4F08C060817181072E000C880B990B8E
:107180000E5F1F4FF32DFF763F2E97FF09C090959E
:107190008095709561957F4F8F4F9F4FF0683F2E80
:1071A0002AE030E0A3010E94123D882E861845C0D7
:1071B000853731F4232D2F7EB22E2AE030E025C012
:1071C000932D997FB92E8F36C1F018F4883579F058
:1071D000B5C0803719F0883721F0B0C0E92FE061E1
:1071E000BE2EB4FE0DC0FB2DF460BF2E09C034FED0
:1071F0000AC0292F2660B22E06C028E030E005C064
:1072000020E130E002C020E132E0F801B7FE07C023
:1072100060817181828193810C5F1F4F06C0608104
:10722000718180E090E00E5F1F4FA3010E94123D2C
:10723000882E8618FB2DFF773F2E36FE0DC0232D9E
:107240002E7FA22E891458F434FE0BC032FC09C0E4
:10725000832D8E7EA82E05C0B82CA32C03C0B82C7D
:1072600001C0B92CA4FE0FC0FE01E80DF11D808104
:10727000803321F49A2D997EA92E09C0A2FE06C062
:10728000B394B39404C08A2D867809F0B394A3FC18
:1072900011C0A0FE06C0B21488F4280C922C9B18D2
:1072A0000EC0B21460F4B60180E290E00E94BD3CD2
:1072B000B394F7CFB21418F42B1802C0982C212CD9
:1072C000A4FE10C0B60180E390E00E94BD3CA2FE87
:1072D00017C0A1FC03C088E790E002C088E590E0F9
:1072E000B6010CC08A2D867859F0A1FE02C08BE24F
:1072F00001C080E2A7FC8DE2B60190E00E94BD3C97
:10730000891438F4B60180E390E00E94BD3C9A9461
:10731000F7CF8A94F301E80DF11D8081B60190E06A
:107320000E94BD3C8110F5CF222009F442CEB60167
:1073300080E290E00E94BD3C2A94F6CFF60186815F
:10734000978102C08FEF9FEF2B96E2E10C94E73418
:1073500020FD09C0FC0123FD05C022FF02C073838C
:10736000628351834083089544FD17C046FD17C0D2
:10737000AB01BC01DA01FB01AA0FBB1FEE1FFF1F0F
:107380001094D1F74A0F5B1F6E1F7F1FCB01BA010C
:10739000660F771F881F991F09C033E001C034E0D2
:1073A000660F771F881F991F3150D1F7620F711D2B
:1073B000811D911D08950F931F93CF93DF938C012F
:1073C000C8010E947F3CEC0197FD08C00E94553C1B
:1073D000892BB1F7B801CE010E94F93CCE01DF91B3
:1073E000CF911F910F9108958F929F92AF92BF926C
:1073F000EF92FF920F931F93CF93DF938C01D62FC1
:107400007A01B22E0E947F3C9C0133272B3231053A
:1074100031F02D32310561F48B2D8068B82ED150BA
:1074200011F480E068C0C8010E947F3C97FDF9CF4D
:10743000CB2DCD7F2B2D207309F58033F9F4AA24B1
:10744000AA94AD0E09F443C0C8010E947F3C97FD89
:107450003EC09C012F7D33272835310549F4C26495
:10746000D250A9F1C8010E947F3C97FF07C02FC0EE
:10747000B6FE02C0C26001C0C261DA2D812C912C1F
:10748000540120ED280F283080F0C4FF04C0B8015B
:107490000E94F93C19C02A3040F0C6FFF8CF2F7D7A
:1074A0003FEE320F363098F727504C2FC501B4010C
:1074B0000E94B4394B015C01C260D15059F0C8013F
:1074C0000E947F3C97FFDDCFC1FD04C0AACF812C75
:1074D000912C5401C7FF08C0B094A094909480945C
:1074E000811C911CA11CB11C2C2FB501A401C7014A
:1074F0000E94A83981E0DF91CF911F910F91FF90F9
:10750000EF90BF90AF909F908F900895A0E2B0E071
:10751000ECE8FAE30C94CE345C01962E7A01F90182
:107520008E010F5F1F4F680180E2D8011D928A957E
:10753000E9F7D50113968C9080E090E0612C712CD6
:1075400030E061E070E083FC259183FE21918F01A2
:10755000522E211103C080E090E092C02E3511F42C
:10756000009751F1432F50E0481759073CF42D354F
:1075700059F12D3219F4772009F103C0772009F46D
:107580006AC0452D469546954695D601A40FB11D76
:10759000452D47708B0102C0000F111F4A95E2F77D
:1075A000A8015C91452B4C93651459F0561410F4C6
:1075B0005394E7CF5A94E5CF31E004C07724739415
:1075C00001C0712C0196BFCF772019F08E818062A7
:1075D0008E83311103C08824839417C0F6019E0165
:1075E0002F5D3F4F8081809581932E173F07D1F704
:1075F000F2CFE114F10429F0D7018C93F701319611
:107600007F019A94812C9920F9F0C5010E947F3C5A
:1076100097FD18C0FC01FF2723E0F595E7952A9513
:10762000E1F7EC0DFD1D208130E0AC0147705527DE
:1076300002C0359527954A95E2F720FDDACFB501CE
:107640000E94F93C811087CFE114F10411F0D701B9
:107650001C92C80115C0422F469546954695D60105
:10766000A40FB11D422F47708B0102C0000F111FE4
:107670004A95E2F7A8015C91452B4C93622EA2CF6C
:10768000A096EFE00C94EA34A0E0B0E0EAE4FBE37B
:107690000C94CE346C01EB015A01FC011782168266
:1076A000512CF601E380FE01E3FC8591E3FE81911C
:1076B000182FEF01882309F4EEC090E00E94553C9A
:1076C000892B21F0C6010E94DB39EBCF153241F442
:1076D000FE01E3FC1591E3FE1191EF01153281F4F7
:1076E000C6010E947F3C97FDD4C0412F50E09C0111
:1076F000332724173507A9F2B6010E94F93CCBC005
:107700001A3239F4E3FC1591E3FE1191EF0101E027
:1077100001C000E0F12C20ED210F2A3080F402603E
:107720006F2D70E080E090E040E20E94B439F62EC8
:10773000FE01E3FC1591E3FE1191EF01ECCF01FF97
:1077400003C0F11003C0A7C0FF24FA94183619F043
:107750001C3651F010C0FE01E3FC1591E3FE1191BF
:10776000EF01183641F408600460FE01E3FC159156
:10777000E3FE1191EF01112309F48DC0612F70E038
:1077800088EE90E00E945E3C892B09F484C000FDE5
:1077900007C0F50180809180C50102965C0102C09E
:1077A000812C912C1E3651F4F6014681578160E000
:1077B00070E0202FC4010E94A83973CF1336A9F4BA
:1077C00001FD02C0FF24F394C6010E947F3C97FD97
:1077D00060C08114910429F0F4018083C4010196F2
:1077E0004C01FA94F110F0CF50C01B3559F49E01B2
:1077F000A4016F2DC6010E94863AEC01892B09F085
:1078000044C03EC0C6010E94DB3997FD42C01F360E
:1078100061F128F4143639F1193651F128C01337C3
:1078200071F0153701F123C08114910429F0F4019E
:107830006082C40101964C01FA94FF2071F0C601E8
:107840000E947F3C3C0197FD08C00E94553C892B5B
:1078500059F3B601C3010E94F93C81149104A9F0C7
:10786000F401108212C0006203C0006101C0006414
:10787000202FA4016F2DC6010E94F439811105C08B
:10788000F6018381807329F406C000FD0ACF53946A
:1078900008CF552019F0852D90E002C08FEF9FEFA3
:1078A000CDB7DEB7EFE00C94EA3491110C94703D43
:1078B000803219F089508550C8F70895FC01059071
:1078C000061621F00020D9F7C00108953197CF01A5
:1078D0000895FC010590615070400110D8F7809523
:1078E00090958E0F9F1F0895FC016150704001908C
:1078F0000110D8F7809590958E0F9F1F0895CF9314
:10790000DF93EC012B8120FF33C026FF0AC02F7BC1
:107910002B838E819F8101969F838E838A8190E045
:1079200029C022FF0FC0E881F9818081082E000C58
:10793000990B009719F420622B831AC03196F983B2
:10794000E8830EC0EA85FB85099597FF09C02B8166
:10795000019611F080E201C080E1822B8B8308C088
:107960002E813F812F5F3F4F3F832E83992702C097
:107970008FEF9FEFDF91CF9108950F931F93CF93D8
:10798000DF93FB01238121FD03C08FEF9FEF2CC00C
:1079900022FF16C046815781248135814217530743
:1079A00044F4A081B1819D012F5F3F4F318320833B
:1079B0008C93268137812F5F3F4F3783268314C0F6
:1079C0008B01EC01FB010084F185E02D0995892BE9
:1079D000E1F6D80116968D919C911797019617960E
:1079E0009C938E931697CE01DF91CF911F910F91AB
:1079F0000895FB01238120FF12C026FD10C08F3F98
:107A00003FEF930761F082832F7D206423832681DB
:107A100037812150310937832683992708958FEFC5
:107A20009FEF0895FA01AA27283051F1203181F102
:107A3000E8946F936E7F6E5F7F4F8F4F9F4FAF4F76
:107A4000B1E03ED0B4E03CD0670F781F891F9A1F89
:107A5000A11D680F791F8A1F911DA11D6A0F711D3D
:107A6000811D911DA11D20D009F468943F912AE049
:107A7000269F11243019305D3193DEF6CF01089531
:107A8000462F4770405D4193B3E00FD0C9F7F6CF62
:107A9000462F4F70405D4A3318F0495D31FD40522A
:107AA000419302D0A9F7EACFB4E0A69597958795C0
:107AB00077956795BA95C9F700976105710508959F
:107AC0009B01AC010A2E069457954795379527954B
:107AD000BA95C9F7620F731F841F951FA01D0895E3
:107AE000992788270895F999FECF92BD81BDF89A0C
:107AF000992780B50895A6E1B0E044E050E00C94E9
:107B0000AD3DA8E1B0E042E050E00C94AD3D262F41
:107B1000F999FECF92BD81BDF89A019700B4021683
:107B200039F01FBA20BD0FB6F894FA9AF99A0FBE31
:107B300008950396272F0E94883D0E94873D252F98
:107B40000E94883D242F0C94883D0196272F0E9487
:107B5000883D0C94873DDC01CB01FC01F999FECFF7
:107B600006C0F2BDE1BDF89A319600B40D924150C5
:0A7B70005040B8F70895F894FFCFD5
:107B7A003C02FF2901A4251E040AF92392030747A0
:107B8A0024F20208CF24A2020430268E0201010345
:107B9A0003030303030303030303030103030303AD
:107BAA000303030303030303030307F00040010174
:107BBA0005012F000000000000000000000000FF87
:107BCA00FF4001F00001000000537461727400501C
:107BDA006175736500547572626F00457869740047
:107BEA00526F74617465005363726F6C6C00426FFC
:107BFA006F744431003130353000426C616E6B0075
:107C0A0053617665496D005361766500546F700063
:107C1A0050726576004F4B004E657874004C617364
:107C2A00740044303A0044313A3C656D7074793ED0
:107C3A0020202020200044323A3C656D7074793E41
:107C4A0020202020200044333A3C656D7074793E30
:107C5A0020202020200044343A3C656D7074793E1F
:107C6A00202020202000546170653A004E6577007C
:087C7A003E3E3E004366670038
:00000001FF
